 iterreachobj002

 Timestamp is 4b1a4962 (reproducible build file hash)

 Preferred load address is 0000000180000000

 Start         Length     Name                   Class
 0001:00000000 00004130H .text$mn                CODE
 0001:00004130 00000036H .text$mn$00             CODE
 0001:00004166 00000092H .text$x                 CODE
 0002:00000000 000001c8H .idata$5                DATA
 0002:000001c8 00000038H .00cfg                  DATA
 0002:00000200 00000008H .CRT$XCA                DATA
 0002:00000208 00000008H .CRT$XCZ                DATA
 0002:00000210 00000008H .CRT$XIA                DATA
 0002:00000218 00000008H .CRT$XIC                DATA
 0002:00000220 00000008H .CRT$XIZ                DATA
 0002:00000228 00000008H .CRT$XLA                DATA
 0002:00000230 00000008H .CRT$XLZ                DATA
 0002:00000238 00000008H .CRT$XPA                DATA
 0002:00000240 00000008H .CRT$XPZ                DATA
 0002:00000248 00000008H .CRT$XTA                DATA
 0002:00000250 00000010H .CRT$XTZ                DATA
 0002:00000258 00000000H .gehcont$y              DATA
 0002:00000258 00000000H .gfids$y                DATA
 0002:00000260 000028a0H .rdata                  DATA
 0002:00002b00 00000000H .rdata$CastGuardVftablesA DATA
 0002:00002b00 00000000H .rdata$CastGuardVftablesC DATA
 0002:00002b00 00000028H .rdata$T                DATA
 0002:00002b28 00000188H .rdata$voltmd           DATA
 0002:00002cb0 00000320H .rdata$zzzdbg           DATA
 0002:00002fd0 00000008H .rtc$IAA                DATA
 0002:00002fd8 00000008H .rtc$IZZ                DATA
 0002:00002fe0 00000008H .rtc$TAA                DATA
 0002:00002fe8 00000008H .rtc$TZZ                DATA
 0002:00002ff0 00000004H .tls                    DATA
 0002:00002ff4 00000004H .tls$                   DATA
 0002:00002ff8 00000008H .tls$ZZZ                DATA
 0002:00003000 00000330H .xdata                  DATA
 0002:00003330 00000368H .edata                  DATA
 0002:00003698 0000008cH .idata$2                DATA
 0002:00003724 00000014H .idata$3                DATA
 0002:00003738 000001c8H .idata$4                DATA
 0002:00003900 00000486H .idata$6                DATA
 0003:00000000 00000080H .data                   DATA
 0003:00000080 0001b3b8H .bss                    DATA
 0004:00000000 000003fcH .pdata                  DATA

  Address         Publics by Value              Rva+Base               Lib:Object

 0000:00000000       __AbsoluteZero             0000000000000000     <absolute>
 0000:00000000       ___safe_se_handler_count   0000000000000000     <absolute>
 0000:00000000       ___safe_se_handler_table   0000000000000000     <absolute>
 0000:00000000       __arm64x_extra_rfe_table   0000000000000000     <absolute>
 0000:00000000       __arm64x_extra_rfe_table_size 0000000000000000     <absolute>
 0000:00000000       __arm64x_native_entrypoint 0000000000000000     <absolute>
 0000:00000000       __arm64x_redirection_metadata 0000000000000000     <absolute>
 0000:00000000       __arm64x_redirection_metadata_count 0000000000000000     <absolute>
 0000:00000000       __dynamic_value_reloc_table 0000000000000000     <absolute>
 0000:00000000       __enclave_config           0000000000000000     <absolute>
 0000:00000000       __guard_check_icall_a64n_fptr 0000000000000000     <absolute>
 0000:00000000       __guard_eh_cont_count      0000000000000000     <absolute>
 0000:00000000       __guard_eh_cont_table      0000000000000000     <absolute>
 0000:00000000       __guard_fids_count         0000000000000000     <absolute>
 0000:00000000       __guard_fids_table         0000000000000000     <absolute>
 0000:00000000       __guard_iat_count          0000000000000000     <absolute>
 0000:00000000       __guard_iat_table          0000000000000000     <absolute>
 0000:00000000       __guard_longjmp_count      0000000000000000     <absolute>
 0000:00000000       __guard_longjmp_table      0000000000000000     <absolute>
 0000:00000000       __hybrid_auxiliary_iat     0000000000000000     <absolute>
 0000:00000000       __hybrid_auxiliary_iat_copy 0000000000000000     <absolute>
 0000:00000000       __hybrid_code_map          0000000000000000     <absolute>
 0000:00000000       __hybrid_code_map_count    0000000000000000     <absolute>
 0000:00000000       __x64_code_ranges_to_entry_points 0000000000000000     <absolute>
 0000:00000000       __x64_code_ranges_to_entry_points_count 0000000000000000     <absolute>
 0000:00000100       __guard_flags              0000000000000100     <absolute>
 0000:00000000       __ImageBase                0000000180000000     <linker-defined>
 0001:00000000       ?NewObject@JNIEnv_@@QEAAPEAV_jobject@@PEAV_jclass@@PEAU_jmethodID@@ZZ 0000000180001000 f i libiterreachobj002.obj
 0001:00000024       ?SetEventNotificationMode@_jvmtiEnv@@QEAA?AW4jvmtiError@@W4jvmtiEventMode@@W4jvmtiEvent@@PEAV_jobject@@ZZ 0000000180001024 f i libiterreachobj002.obj
 0001:0000002c       ?TranslateError@@YAPEBDW4jvmtiError@@@Z 000000018000102c f   libiterreachobj002.obj
 0001:000002e4       ?nsk_jni_check_exception@@YAHPEAUJNIEnv_@@QEBDH@Z 00000001800012e4 f   libiterreachobj002.obj
 0001:00000428       ?nsk_jni_lverify@@YAHHPEAUJNIEnv_@@HQEBDH1ZZ 0000000180001428 f   libiterreachobj002.obj
 0001:000004c8       Agent_Initialize           00000001800014c8 f   libiterreachobj002.obj
 0001:00000870       Agent_OnAttach             0000000180001870 f   libiterreachobj002.obj
 0001:00000870       Agent_OnLoad               0000000180001870 f   libiterreachobj002.obj
 0001:00000878       Java_nsk_jvmti_unit_FollowReferences_FollowRefObjects_addRefToVerify 0000000180001878 f   libiterreachobj002.obj
 0001:00000a34       Java_nsk_jvmti_unit_FollowReferences_FollowRefObjects_getTag 0000000180001a34 f   libiterreachobj002.obj
 0001:00000af0       Java_nsk_jvmti_unit_FollowReferences_FollowRefObjects_resetRefsToVerify 0000000180001af0 f   libiterreachobj002.obj
 0001:00000af8       Java_nsk_jvmti_unit_FollowReferences_FollowRefObjects_resetTags 0000000180001af8 f   libiterreachobj002.obj
 0001:00000b3c       Java_nsk_jvmti_unit_FollowReferences_FollowRefObjects_setTag 0000000180001b3c f   libiterreachobj002.obj
 0001:00000d88       Java_nsk_share_jvmti_ArgumentHandler_getAgentOptionsString 0000000180001d88 f   libiterreachobj002.obj
 0001:00000e34       Java_nsk_share_jvmti_DebugeeClass_checkStatus 0000000180001e34 f   libiterreachobj002.obj
 0001:00000ebc       Java_nsk_share_jvmti_DebugeeClass_resetAgentData 0000000180001ebc f   libiterreachobj002.obj
 0001:00000f1c       Java_nsk_share_jvmti_RedefineAgent_agentStatus 0000000180001f1c f   libiterreachobj002.obj
 0001:00000f28       Java_nsk_share_jvmti_RedefineAgent_isRedefined 0000000180001f28 f   libiterreachobj002.obj
 0001:00000f34       Java_nsk_share_jvmti_RedefineAgent_redefineAttempted 0000000180001f34 f   libiterreachobj002.obj
 0001:00000f40       MA_checkStatus             0000000180001f40 f   libiterreachobj002.obj
 0001:00000fe4       ObjectFree                 0000000180001fe4 f   libiterreachobj002.obj
 0001:00000ff4       __local_stdio_printf_options 0000000180001ff4 f i libiterreachobj002.obj
 0001:000019d4       exitOnError                00000001800029d4 f   libiterreachobj002.obj
 0001:00001a88       fprintf                    0000000180002a88 f i libiterreachobj002.obj
 0001:00001acc       heapRootCallbackForFirstObjectsIteration 0000000180002acc f   libiterreachobj002.obj
 0001:00001bf0       heapRootCallbackForSecondObjectsIteration 0000000180002bf0 f   libiterreachobj002.obj
 0001:00001d4c       nsk_complain               0000000180002d4c f   libiterreachobj002.obj
 0001:00001d78       nsk_jvmti_createJVMTIEnv   0000000180002d78 f   libiterreachobj002.obj
 0001:00001ea8       nsk_jvmti_lverify          0000000180002ea8 f   libiterreachobj002.obj
 0001:00001f98       nsk_jvmti_parseOptions     0000000180002f98 f   libiterreachobj002.obj
 0001:000021e8       nsk_jvmti_resetAgentData   00000001800031e8 f   libiterreachobj002.obj
 0001:0000225c       nsk_jvmti_resumeSync       000000018000325c f   libiterreachobj002.obj
 0001:00002300       nsk_jvmti_waitForSync      0000000180003300 f   libiterreachobj002.obj
 0001:00002404       nsk_lcomplain              0000000180003404 f   libiterreachobj002.obj
 0001:00002424       nsk_ldisplay               0000000180003424 f   libiterreachobj002.obj
 0001:00002444       nsk_ltrace                 0000000180003444 f   libiterreachobj002.obj
 0001:00002464       nsk_lvcomplain             0000000180003464 f   libiterreachobj002.obj
 0001:0000261c       nsk_lvdisplay              000000018000361c f   libiterreachobj002.obj
 0001:00002668       nsk_lverify                0000000180003668 f   libiterreachobj002.obj
 0001:000026c4       nsk_lvtrace                00000001800036c4 f   libiterreachobj002.obj
 0001:00002724       nsk_printf                 0000000180003724 f   libiterreachobj002.obj
 0001:0000274c       nsk_vprintf                000000018000374c f   libiterreachobj002.obj
 0001:00002800       objectReferenceCallbackForFirstObjectsIteration 0000000180003800 f   libiterreachobj002.obj
 0001:00002928       objectReferenceCallbackForSecondObjectsIteration 0000000180003928 f   libiterreachobj002.obj
 0001:00002a84       printf                     0000000180003a84 f i libiterreachobj002.obj
 0001:00002ad8       stackReferenceCallbackForFirstObjectsIteration 0000000180003ad8 f   libiterreachobj002.obj
 0001:00002c00       stackReferenceCallbackForSecondObjectsIteration 0000000180003c00 f   libiterreachobj002.obj
 0001:00003208       __raise_securityfailure    0000000180004208 f   MSVCRT:gs_report.obj
 0001:0000323c       __report_gsfailure         000000018000423c f   MSVCRT:gs_report.obj
 0001:0000347c       __GSHandlerCheck           000000018000447c f   MSVCRT:gshandler.obj
 0001:0000349c       __GSHandlerCheckCommon     000000018000449c f   MSVCRT:gshandler.obj
 0001:00003510       __security_check_cookie    0000000180004510 f   MSVCRT:amdsecgs.obj
 0001:00003850       _DllMainCRTStartup         0000000180004850 f   MSVCRT:dll_dllmain.obj
 0001:00003890       __scrt_acquire_startup_lock 0000000180004890 f   MSVCRT:utility.obj
 0001:000038cc       __scrt_dllmain_after_initialize_c 00000001800048cc f   MSVCRT:utility.obj
 0001:00003900       __scrt_dllmain_before_initialize_c 0000000180004900 f   MSVCRT:utility.obj
 0001:00003918       __scrt_dllmain_crt_thread_attach 0000000180004918 f   MSVCRT:utility.obj
 0001:00003940       __scrt_dllmain_crt_thread_detach 0000000180004940 f   MSVCRT:utility.obj
 0001:00003958       __scrt_dllmain_exception_filter 0000000180004958 f   MSVCRT:utility.obj
 0001:000039b8       __scrt_dllmain_uninitialize_c 00000001800049b8 f   MSVCRT:utility.obj
 0001:000039e8       __scrt_dllmain_uninitialize_critical 00000001800049e8 f   MSVCRT:utility.obj
 0001:000039fc       __scrt_initialize_crt      00000001800049fc f   MSVCRT:utility.obj
 0001:00003a48       __scrt_initialize_onexit_tables 0000000180004a48 f   MSVCRT:utility.obj
 0001:00003ad4       __scrt_is_nonwritable_in_current_image 0000000180004ad4 f   MSVCRT:utility.obj
 0001:00003b6c       __scrt_release_startup_lock 0000000180004b6c f   MSVCRT:utility.obj
 0001:00003b90       __scrt_uninitialize_crt    0000000180004b90 f   MSVCRT:utility.obj
 0001:00003bbc       _onexit                    0000000180004bbc f   MSVCRT:utility.obj
 0001:00003bf8       atexit                     0000000180004bf8 f   MSVCRT:utility.obj
 0001:00003c10       __crt_debugger_hook        0000000180004c10 f   MSVCRT:utility_desktop.obj
 0001:00003c18       __scrt_fastfail            0000000180004c18 f   MSVCRT:utility_desktop.obj
 0001:00003d64       _guard_check_icall_nop     0000000180004d64 f i MSVCRT:guard_support.obj
 0001:00003d68       __security_init_cookie     0000000180004d68 f   MSVCRT:gs_support.obj
 0001:00003e14       DllMain                    0000000180004e14 f   MSVCRT:dll_dllmain_stub.obj
 0001:00003e38       ?__scrt_initialize_type_info@@YAXXZ 0000000180004e38 f   MSVCRT:tncleanup.obj
 0001:00003e48       ?__scrt_uninitialize_type_info@@YAXXZ 0000000180004e48 f   MSVCRT:tncleanup.obj
 0001:00003e54       __local_stdio_scanf_options 0000000180004e54 f i MSVCRT:default_local_stdio_options.obj
 0001:00003e5c       __scrt_initialize_default_local_stdio_options 0000000180004e5c f   MSVCRT:default_local_stdio_options.obj
 0001:00003e78       __scrt_get_dyn_tls_init_callback 0000000180004e78 f   MSVCRT:dyn_tls_init.obj
 0001:00003e80       _RTC_Initialize            0000000180004e80 f   MSVCRT:initsect.obj
 0001:00003ebc       _RTC_Terminate             0000000180004ebc f   MSVCRT:initsect.obj
 0001:00003ef8       __isa_available_init       0000000180004ef8 f   MSVCRT:cpu_disp.obj
 0001:000040a4       _get_startup_argv_mode     00000001800050a4 f   MSVCRT:argv_mode.obj
 0001:000040ac       __scrt_is_ucrt_dll_in_use  00000001800050ac f   MSVCRT:ucrt_detection.obj
 0001:000040c0       memcpy                     00000001800050c0 f   vcruntime:VCRUNTIME140.dll
 0001:000040c6       memset                     00000001800050c6 f   vcruntime:VCRUNTIME140.dll
 0001:000040cc       strchr                     00000001800050cc f   vcruntime:VCRUNTIME140.dll
 0001:000040d2       __C_specific_handler       00000001800050d2 f   vcruntime:VCRUNTIME140.dll
 0001:000040d8       __std_type_info_destroy_list 00000001800050d8 f   vcruntime:VCRUNTIME140.dll
 0001:000040de       strcmp                     00000001800050de f   ucrt:api-ms-win-crt-string-l1-1-0.dll
 0001:000040e4       strlen                     00000001800050e4 f   ucrt:api-ms-win-crt-string-l1-1-0.dll
 0001:000040ea       _initterm                  00000001800050ea f   ucrt:api-ms-win-crt-runtime-l1-1-0.dll
 0001:000040f0       _initterm_e                00000001800050f0 f   ucrt:api-ms-win-crt-runtime-l1-1-0.dll
 0001:000040f6       _seh_filter_dll            00000001800050f6 f   ucrt:api-ms-win-crt-runtime-l1-1-0.dll
 0001:000040fc       _configure_narrow_argv     00000001800050fc f   ucrt:api-ms-win-crt-runtime-l1-1-0.dll
 0001:00004102       _initialize_narrow_environment 0000000180005102 f   ucrt:api-ms-win-crt-runtime-l1-1-0.dll
 0001:00004108       _initialize_onexit_table   0000000180005108 f   ucrt:api-ms-win-crt-runtime-l1-1-0.dll
 0001:0000410e       _register_onexit_function  000000018000510e f   ucrt:api-ms-win-crt-runtime-l1-1-0.dll
 0001:00004114       _execute_onexit_table      0000000180005114 f   ucrt:api-ms-win-crt-runtime-l1-1-0.dll
 0001:0000411a       _crt_atexit                000000018000511a f   ucrt:api-ms-win-crt-runtime-l1-1-0.dll
 0001:00004120       _cexit                     0000000180005120 f   ucrt:api-ms-win-crt-runtime-l1-1-0.dll
 0001:00004128       __acrt_initialize          0000000180005128 f   MSVCRT:ucrt_stubs.obj
 0001:00004128       __acrt_thread_attach       0000000180005128 f   MSVCRT:ucrt_stubs.obj
 0001:00004128       __acrt_thread_detach       0000000180005128 f   MSVCRT:ucrt_stubs.obj
 0001:00004128       __acrt_uninitialize        0000000180005128 f   MSVCRT:ucrt_stubs.obj
 0001:00004128       __acrt_uninitialize_critical 0000000180005128 f   MSVCRT:ucrt_stubs.obj
 0001:00004128       __scrt_stub_for_acrt_initialize 0000000180005128 f   MSVCRT:ucrt_stubs.obj
 0001:00004128       __scrt_stub_for_acrt_thread_attach 0000000180005128 f   MSVCRT:ucrt_stubs.obj
 0001:00004128       __scrt_stub_for_acrt_thread_detach 0000000180005128 f   MSVCRT:ucrt_stubs.obj
 0001:00004128       __scrt_stub_for_acrt_uninitialize 0000000180005128 f   MSVCRT:ucrt_stubs.obj
 0001:00004128       __scrt_stub_for_acrt_uninitialize_critical 0000000180005128 f   MSVCRT:ucrt_stubs.obj
 0001:00004128       __vcrt_initialize          0000000180005128 f   MSVCRT:ucrt_stubs.obj
 0001:00004128       __vcrt_thread_attach       0000000180005128 f   MSVCRT:ucrt_stubs.obj
 0001:00004128       __vcrt_thread_detach       0000000180005128 f   MSVCRT:ucrt_stubs.obj
 0001:00004128       __vcrt_uninitialize        0000000180005128 f   MSVCRT:ucrt_stubs.obj
 0001:00004128       __vcrt_uninitialize_critical 0000000180005128 f   MSVCRT:ucrt_stubs.obj
 0001:0000412c       __scrt_stub_for_is_c_termination_complete 000000018000512c f   MSVCRT:ucrt_stubs.obj
 0001:0000412c       _is_c_termination_complete 000000018000512c f   MSVCRT:ucrt_stubs.obj
 0001:00004140       _guard_dispatch_icall_nop  0000000180005140 f   MSVCRT:guard_dispatch.obj
 0001:00004160       _guard_xfg_dispatch_icall_nop 0000000180005160 f   MSVCRT:guard_xfg_dispatch.obj
 0002:00000000       __imp_RtlCaptureContext    0000000180006000     kernel32:KERNEL32.dll
 0002:00000008       __imp_RtlLookupFunctionEntry 0000000180006008     kernel32:KERNEL32.dll
 0002:00000010       __imp_RtlVirtualUnwind     0000000180006010     kernel32:KERNEL32.dll
 0002:00000018       __imp_UnhandledExceptionFilter 0000000180006018     kernel32:KERNEL32.dll
 0002:00000020       __imp_SetUnhandledExceptionFilter 0000000180006020     kernel32:KERNEL32.dll
 0002:00000028       __imp_GetCurrentProcess    0000000180006028     kernel32:KERNEL32.dll
 0002:00000030       __imp_TerminateProcess     0000000180006030     kernel32:KERNEL32.dll
 0002:00000038       __imp_IsProcessorFeaturePresent 0000000180006038     kernel32:KERNEL32.dll
 0002:00000040       __imp_CloseHandle          0000000180006040     kernel32:KERNEL32.dll
 0002:00000048       __imp_InitializeCriticalSectionAndSpinCount 0000000180006048     kernel32:KERNEL32.dll
 0002:00000050       __imp_DeleteCriticalSection 0000000180006050     kernel32:KERNEL32.dll
 0002:00000058       __imp_CreateEventW         0000000180006058     kernel32:KERNEL32.dll
 0002:00000060       __imp_GetModuleHandleW     0000000180006060     kernel32:KERNEL32.dll
 0002:00000068       __imp_GetProcAddress       0000000180006068     kernel32:KERNEL32.dll
 0002:00000070       __imp_IsDebuggerPresent    0000000180006070     kernel32:KERNEL32.dll
 0002:00000078       __imp_QueryPerformanceCounter 0000000180006078     kernel32:KERNEL32.dll
 0002:00000080       __imp_GetCurrentProcessId  0000000180006080     kernel32:KERNEL32.dll
 0002:00000088       __imp_GetCurrentThreadId   0000000180006088     kernel32:KERNEL32.dll
 0002:00000090       __imp_GetSystemTimeAsFileTime 0000000180006090     kernel32:KERNEL32.dll
 0002:00000098       __imp_DisableThreadLibraryCalls 0000000180006098     kernel32:KERNEL32.dll
 0002:000000a0       __imp_InitializeSListHead  00000001800060a0     kernel32:KERNEL32.dll
 0002:000000a8       \177KERNEL32_NULL_THUNK_DATA 00000001800060a8     kernel32:KERNEL32.dll
 0002:000000b0       __imp_memcpy               00000001800060b0     vcruntime:VCRUNTIME140.dll
 0002:000000b8       __imp_memset               00000001800060b8     vcruntime:VCRUNTIME140.dll
 0002:000000c0       __imp_strchr               00000001800060c0     vcruntime:VCRUNTIME140.dll
 0002:000000c8       __imp___C_specific_handler 00000001800060c8     vcruntime:VCRUNTIME140.dll
 0002:000000d0       __imp___std_type_info_destroy_list 00000001800060d0     vcruntime:VCRUNTIME140.dll
 0002:000000d8       \177VCRUNTIME140_NULL_THUNK_DATA 00000001800060d8     vcruntime:VCRUNTIME140.dll
 0002:000000e0       __imp_strtol               00000001800060e0     ucrt:api-ms-win-crt-convert-l1-1-0.dll
 0002:000000e8       \177api-ms-win-crt-convert-l1-1-0_NULL_THUNK_DATA 00000001800060e8     ucrt:api-ms-win-crt-convert-l1-1-0.dll
 0002:000000f0       __imp_malloc               00000001800060f0     ucrt:api-ms-win-crt-heap-l1-1-0.dll
 0002:000000f8       __imp_free                 00000001800060f8     ucrt:api-ms-win-crt-heap-l1-1-0.dll
 0002:00000100       \177api-ms-win-crt-heap-l1-1-0_NULL_THUNK_DATA 0000000180006100     ucrt:api-ms-win-crt-heap-l1-1-0.dll
 0002:00000108       __imp__errno               0000000180006108     ucrt:api-ms-win-crt-runtime-l1-1-0.dll
 0002:00000110       __imp_exit                 0000000180006110     ucrt:api-ms-win-crt-runtime-l1-1-0.dll
 0002:00000118       __imp__cexit               0000000180006118     ucrt:api-ms-win-crt-runtime-l1-1-0.dll
 0002:00000120       __imp__crt_atexit          0000000180006120     ucrt:api-ms-win-crt-runtime-l1-1-0.dll
 0002:00000128       __imp__execute_onexit_table 0000000180006128     ucrt:api-ms-win-crt-runtime-l1-1-0.dll
 0002:00000130       __imp__register_onexit_function 0000000180006130     ucrt:api-ms-win-crt-runtime-l1-1-0.dll
 0002:00000138       __imp__initialize_onexit_table 0000000180006138     ucrt:api-ms-win-crt-runtime-l1-1-0.dll
 0002:00000140       __imp__initialize_narrow_environment 0000000180006140     ucrt:api-ms-win-crt-runtime-l1-1-0.dll
 0002:00000148       __imp__configure_narrow_argv 0000000180006148     ucrt:api-ms-win-crt-runtime-l1-1-0.dll
 0002:00000150       __imp__seh_filter_dll      0000000180006150     ucrt:api-ms-win-crt-runtime-l1-1-0.dll
 0002:00000158       __imp__initterm_e          0000000180006158     ucrt:api-ms-win-crt-runtime-l1-1-0.dll
 0002:00000160       __imp__initterm            0000000180006160     ucrt:api-ms-win-crt-runtime-l1-1-0.dll
 0002:00000168       \177api-ms-win-crt-runtime-l1-1-0_NULL_THUNK_DATA 0000000180006168     ucrt:api-ms-win-crt-runtime-l1-1-0.dll
 0002:00000170       __imp___acrt_iob_func      0000000180006170     ucrt:api-ms-win-crt-stdio-l1-1-0.dll
 0002:00000178       __imp_fflush               0000000180006178     ucrt:api-ms-win-crt-stdio-l1-1-0.dll
 0002:00000180       __imp___stdio_common_vsprintf 0000000180006180     ucrt:api-ms-win-crt-stdio-l1-1-0.dll
 0002:00000188       __imp___stdio_common_vfprintf 0000000180006188     ucrt:api-ms-win-crt-stdio-l1-1-0.dll
 0002:00000190       \177api-ms-win-crt-stdio-l1-1-0_NULL_THUNK_DATA 0000000180006190     ucrt:api-ms-win-crt-stdio-l1-1-0.dll
 0002:00000198       __imp_strcmp               0000000180006198     ucrt:api-ms-win-crt-string-l1-1-0.dll
 0002:000001a0       __imp__strdup              00000001800061a0     ucrt:api-ms-win-crt-string-l1-1-0.dll
 0002:000001a0       __imp_strdup               00000001800061a0     ucrt:api-ms-win-crt-string-l1-1-0.dll
 0002:000001a8       __imp_strlen               00000001800061a8     ucrt:api-ms-win-crt-string-l1-1-0.dll
 0002:000001b0       __imp_strpbrk              00000001800061b0     ucrt:api-ms-win-crt-string-l1-1-0.dll
 0002:000001b8       __imp_strncpy              00000001800061b8     ucrt:api-ms-win-crt-string-l1-1-0.dll
 0002:000001c0       \177api-ms-win-crt-string-l1-1-0_NULL_THUNK_DATA 00000001800061c0     ucrt:api-ms-win-crt-string-l1-1-0.dll
 0002:000001c8       __guard_check_icall_fptr   00000001800061c8     MSVCRT:guard_support.obj
 0002:000001d0       __guard_xfg_check_icall_fptr 00000001800061d0     MSVCRT:guard_support.obj
 0002:000001d8       __guard_dispatch_icall_fptr 00000001800061d8     MSVCRT:guard_support.obj
 0002:000001e0       __guard_xfg_dispatch_icall_fptr 00000001800061e0     MSVCRT:guard_support.obj
 0002:000001e8       __guard_xfg_table_dispatch_icall_fptr 00000001800061e8     MSVCRT:guard_support.obj
 0002:000001f0       __castguard_check_failure_os_handled_fptr 00000001800061f0     MSVCRT:guard_support.obj
 0002:000001f8       __guard_memcpy_fptr        00000001800061f8     vcruntime:softmemtag.obj
 0002:00000200       __xc_a                     0000000180006200     MSVCRT:initializers.obj
 0002:00000208       __xc_z                     0000000180006208     MSVCRT:initializers.obj
 0002:00000210       __xi_a                     0000000180006210     MSVCRT:initializers.obj
 0002:00000220       __xi_z                     0000000180006220     MSVCRT:initializers.obj
 0002:00000228       __xl_a                     0000000180006228     MSVCRT:tlssup.obj
 0002:00000230       __xl_z                     0000000180006230     MSVCRT:tlssup.obj
 0002:00000238       __xp_a                     0000000180006238     MSVCRT:initializers.obj
 0002:00000240       __xp_z                     0000000180006240     MSVCRT:initializers.obj
 0002:00000248       __xt_a                     0000000180006248     MSVCRT:initializers.obj
 0002:00000250       __xt_z                     0000000180006250     MSVCRT:initializers.obj
 0002:00000260       g_refKindStr               0000000180006260     libiterreachobj002.obj
 0002:00000410       ??_C@_09BPLDFGCI@unknown_0@ 0000000180006410     libiterreachobj002.obj
 0002:00000420       ??_C@_0BL@FPNMECJD@JVMTI_HEAP_REFERENCE_CLASS@ 0000000180006420     libiterreachobj002.obj
 0002:00000440       ??_C@_0BL@FKGKKLNM@JVMTI_HEAP_REFERENCE_FIELD@ 0000000180006440     libiterreachobj002.obj
 0002:00000460       ??_C@_0CD@CAEHCFJF@JVMTI_HEAP_REFERENCE_ARRAY_ELEM@ 0000000180006460     libiterreachobj002.obj
 0002:00000488       ??_C@_0CC@DNEBMCNK@JVMTI_HEAP_REFERENCE_CLASS_LOAD@ 0000000180006488     libiterreachobj002.obj
 0002:000004b0       ??_C@_0BN@CJMIPEBB@JVMTI_HEAP_REFERENCE_SIGNERS@ 00000001800064b0     libiterreachobj002.obj
 0002:000004d0       ??_C@_0CH@HBOIDPEB@JVMTI_HEAP_REFERENCE_PROTECTION@ 00000001800064d0     libiterreachobj002.obj
 0002:000004f8       ??_C@_0BP@MDKGDGKL@JVMTI_HEAP_REFERENCE_INTERFACE@ 00000001800064f8     libiterreachobj002.obj
 0002:00000518       ??_C@_0CC@JJMIHNJH@JVMTI_HEAP_REFERENCE_STATIC_FIE@ 0000000180006518     libiterreachobj002.obj
 0002:00000540       ??_C@_0CD@IDHEEGID@JVMTI_HEAP_REFERENCE_CONSTANT_P@ 0000000180006540     libiterreachobj002.obj
 0002:00000568       ??_C@_0CA@EFFCHNG@JVMTI_HEAP_REFERENCE_SUPERCLASS@ 0000000180006568     libiterreachobj002.obj
 0002:00000588       ??_C@_0L@PCDFHGCJ@unknown_11@ 0000000180006588     libiterreachobj002.obj
 0002:00000598       ??_C@_0L@NJBICFOK@unknown_12@ 0000000180006598     libiterreachobj002.obj
 0002:000005a8       ??_C@_0L@MAADBEKL@unknown_13@ 00000001800065a8     libiterreachobj002.obj
 0002:000005b8       ??_C@_0L@IPECICGM@unknown_14@ 00000001800065b8     libiterreachobj002.obj
 0002:000005c8       ??_C@_0L@JGFJLDCN@unknown_15@ 00000001800065c8     libiterreachobj002.obj
 0002:000005d8       ??_C@_0L@LNHEOAOO@unknown_16@ 00000001800065d8     libiterreachobj002.obj
 0002:000005e8       ??_C@_0L@KEGPNBKP@unknown_17@ 00000001800065e8     libiterreachobj002.obj
 0002:000005f8       ??_C@_0L@CDPHMNGA@unknown_18@ 00000001800065f8     libiterreachobj002.obj
 0002:00000608       ??_C@_0L@DKOMPMCB@unknown_19@ 0000000180006608     libiterreachobj002.obj
 0002:00000618       ??_C@_0L@OJGIPJDB@unknown_20@ 0000000180006618     libiterreachobj002.obj
 0002:00000628       ??_C@_0CA@KAOFNDEM@JVMTI_HEAP_REFERENCE_JNI_GLOBAL@ 0000000180006628     libiterreachobj002.obj
 0002:00000648       ??_C@_0CC@HPFAJBK@JVMTI_HEAP_REFERENCE_SYSTEM_CLA@ 0000000180006648     libiterreachobj002.obj
 0002:00000670       ??_C@_0BN@FDEGFOHC@JVMTI_HEAP_REFERENCE_MONITOR@ 0000000180006670     libiterreachobj002.obj
 0002:00000690       ??_C@_0CB@HKIBCMAJ@JVMTI_HEAP_REFERENCE_STACK_LOCA@ 0000000180006690     libiterreachobj002.obj
 0002:000006b8       ??_C@_0BP@EAACMMOE@JVMTI_HEAP_REFERENCE_JNI_LOCAL@ 00000001800066b8     libiterreachobj002.obj
 0002:000006d8       ??_C@_0BM@IJDEOGOE@JVMTI_HEAP_REFERENCE_THREAD@ 00000001800066d8     libiterreachobj002.obj
 0002:000006f8       ??_C@_0BL@EDGPPKC@JVMTI_HEAP_REFERENCE_OTHER@ 00000001800066f8     libiterreachobj002.obj
 0002:00000714       ??_C@_04BCJPDBDA@Code@     0000000180006714     libiterreachobj002.obj
 0002:00000720       ??_C@_0BA@OCLMCFKC@LineNumberTable@ 0000000180006720     libiterreachobj002.obj
 0002:00000730       ??_C@_0BD@CPAEPILC@LocalVariableTable@ 0000000180006730     libiterreachobj002.obj
 0002:00000748       ??_C@_0BH@NMBDNHBD@LocalVariableTypeTable@ 0000000180006748     libiterreachobj002.obj
 0002:00000760       ??_C@_0O@HIHEEDNJ@StackMapTable@ 0000000180006760     libiterreachobj002.obj
 0002:00000770       ??_C@_0L@HCDIAMJG@?9?5?$CFs?0?5?$CFd?3?5@ 0000000180006770     libiterreachobj002.obj
 0002:00000780       ??_C@_0JI@HLPECLFI@?$CD?5?4?4?4?6?$CD?5ERROR?3?5too?5many?5complai@ 0000000180006780     libiterreachobj002.obj
 0002:00000820       ??_C@_0ED@JNEKCCOB@The?5following?5fake?5exception?5st@ 0000000180006820     libiterreachobj002.obj
 0002:00000868       ??_C@_0CN@FCNMDFBH@nsk?4share?4Fake_Exception_for_RU@ 0000000180006868     libiterreachobj002.obj
 0002:00000898       ??_C@_08PGFFNAEI@?$CI?$CFs?3?$CFd?$CJ?5@ 0000000180006898     libiterreachobj002.obj
 0002:000008a8       ??_C@_0DP@IENMAEGI@s?2test?2hotspot?2jtreg?2vmTestbase@ 00000001800068a8     libiterreachobj002.obj
 0002:000008e8       ??_C@_0BL@NDJLFFJB@?7at?5nsk_lvcomplain?$CI?$CFs?3?$CFd?$CJ?6@ 00000001800068e8     libiterreachobj002.obj
 0002:00000908       ??_C@_0BC@JOOKAFKF@?$CD?5ERROR?3?5?$CFs?0?5?$CFd?3?5@ 0000000180006908     libiterreachobj002.obj
 0002:00000920       ??_C@_09KJEAHMEH@?$CD?5ERROR?3?5@ 0000000180006920     libiterreachobj002.obj
 0002:0000092c       ??_C@_02GPIOPFAK@?$DO?$DO@ 000000018000692c     libiterreachobj002.obj
 0002:00000930       ??_C@_02FODMEDOG@?$DM?$DM@ 0000000180006930     libiterreachobj002.obj
 0002:00000934       ??_C@_02DJGKEECL@?4?4@     0000000180006934     libiterreachobj002.obj
 0002:00000938       ??_C@_0O@CJPGJOAF@?9?5?$CFs?0?5?$CFd?3?5?$CFs?5@ 0000000180006938     libiterreachobj002.obj
 0002:00000948       ??_C@_0CB@IAKPDOIC@?$CD?5?5?5verified?5assertion?5is?5FALSE@ 0000000180006948     libiterreachobj002.obj
 0002:00000970       ??_C@_0CO@LGONDEPD@stdout?3?5fflush?5failed?5?9?5err?$DN?$CFd?5@ 0000000180006970     libiterreachobj002.obj
 0002:000009a0       ??_C@_0CO@KBGKJPBD@stderr?3?5fflush?5failed?5?9?5err?$DN?$CFd?5@ 00000001800069a0     libiterreachobj002.obj
 0002:000009d0       ??_C@_0BB@JCNMKLLK@JVMTI_ERROR_NONE@ 00000001800069d0     libiterreachobj002.obj
 0002:000009e8       ??_C@_0BL@LDIMKLPH@JVMTI_ERROR_INVALID_THREAD@ 00000001800069e8     libiterreachobj002.obj
 0002:00000a08       ??_C@_0CB@PJFPAIKJ@JVMTI_ERROR_INVALID_THREAD_GROU@ 0000000180006a08     libiterreachobj002.obj
 0002:00000a30       ??_C@_0BN@LLMKHMNF@JVMTI_ERROR_INVALID_PRIORITY@ 0000000180006a30     libiterreachobj002.obj
 0002:00000a50       ??_C@_0CB@MBOFKAGB@JVMTI_ERROR_THREAD_NOT_SUSPENDE@ 0000000180006a50     libiterreachobj002.obj
 0002:00000a78       ??_C@_0BN@FABOLPBI@JVMTI_ERROR_THREAD_SUSPENDED@ 0000000180006a78     libiterreachobj002.obj
 0002:00000a98       ??_C@_0BN@FDGNOBJM@JVMTI_ERROR_THREAD_NOT_ALIVE@ 0000000180006a98     libiterreachobj002.obj
 0002:00000ab8       ??_C@_0BL@GOBIFKNJ@JVMTI_ERROR_INVALID_OBJECT@ 0000000180006ab8     libiterreachobj002.obj
 0002:00000ad8       ??_C@_0BK@FCMAJPPC@JVMTI_ERROR_INVALID_CLASS@ 0000000180006ad8     libiterreachobj002.obj
 0002:00000af8       ??_C@_0BP@IKLLBKEB@JVMTI_ERROR_CLASS_NOT_PREPARED@ 0000000180006af8     libiterreachobj002.obj
 0002:00000b18       ??_C@_0BN@KLPPLKG@JVMTI_ERROR_INVALID_METHODID@ 0000000180006b18     libiterreachobj002.obj
 0002:00000b38       ??_C@_0BN@BCEKOKND@JVMTI_ERROR_INVALID_LOCATION@ 0000000180006b38     libiterreachobj002.obj
 0002:00000b58       ??_C@_0BM@DFDGPME@JVMTI_ERROR_INVALID_FIELDID@ 0000000180006b58     libiterreachobj002.obj
 0002:00000b78       ??_C@_0BL@NELIEPEC@JVMTI_ERROR_NO_MORE_FRAMES@ 0000000180006b78     libiterreachobj002.obj
 0002:00000b98       ??_C@_0BJ@BDBECFDM@JVMTI_ERROR_OPAQUE_FRAME@ 0000000180006b98     libiterreachobj002.obj
 0002:00000bb8       ??_C@_0BK@MIIFNLOB@JVMTI_ERROR_TYPE_MISMATCH@ 0000000180006bb8     libiterreachobj002.obj
 0002:00000bd8       ??_C@_0BJ@HPCAOILC@JVMTI_ERROR_INVALID_SLOT@ 0000000180006bd8     libiterreachobj002.obj
 0002:00000bf8       ??_C@_0BG@CHILOPNI@JVMTI_ERROR_DUPLICATE@ 0000000180006bf8     libiterreachobj002.obj
 0002:00000c10       ??_C@_0BG@DIEMLHKM@JVMTI_ERROR_NOT_FOUND@ 0000000180006c10     libiterreachobj002.obj
 0002:00000c28       ??_C@_0BM@NHMCKHOB@JVMTI_ERROR_INVALID_MONITOR@ 0000000180006c28     libiterreachobj002.obj
 0002:00000c48       ??_C@_0BO@PPEDAJGL@JVMTI_ERROR_NOT_MONITOR_OWNER@ 0000000180006c48     libiterreachobj002.obj
 0002:00000c68       ??_C@_0BG@FCAIPEID@JVMTI_ERROR_INTERRUPT@ 0000000180006c68     libiterreachobj002.obj
 0002:00000c80       ??_C@_0CB@EGDBNKOI@JVMTI_ERROR_INVALID_CLASS_FORMA@ 0000000180006c80     libiterreachobj002.obj
 0002:00000ca8       ??_C@_0CG@DGKOGIAL@JVMTI_ERROR_CIRCULAR_CLASS_DEFI@ 0000000180006ca8     libiterreachobj002.obj
 0002:00000cd0       ??_C@_0BP@ICEALPKC@JVMTI_ERROR_FAILS_VERIFICATION@ 0000000180006cd0     libiterreachobj002.obj
 0002:00000cf0       ??_C@_0DC@JDACLMIO@JVMTI_ERROR_UNSUPPORTED_REDEFIN@ 0000000180006cf0     libiterreachobj002.obj
 0002:00000d28       ??_C@_0DE@GKDKNOMJ@JVMTI_ERROR_UNSUPPORTED_REDEFIN@ 0000000180006d28     libiterreachobj002.obj
 0002:00000d60       ??_C@_0BO@LAFKIOG@JVMTI_ERROR_INVALID_TYPESTATE@ 0000000180006d60     libiterreachobj002.obj
 0002:00000d80       ??_C@_0DH@INDGCLLB@JVMTI_ERROR_UNSUPPORTED_REDEFIN@ 0000000180006d80     libiterreachobj002.obj
 0002:00000db8       ??_C@_0DE@NHEOMMGI@JVMTI_ERROR_UNSUPPORTED_REDEFIN@ 0000000180006db8     libiterreachobj002.obj
 0002:00000df0       ??_C@_0CA@EKPNJOEP@JVMTI_ERROR_UNSUPPORTED_VERSION@ 0000000180006df0     libiterreachobj002.obj
 0002:00000e10       ??_C@_0BN@OFFMAHHL@JVMTI_ERROR_NAMES_DONT_MATCH@ 0000000180006e10     libiterreachobj002.obj
 0002:00000e30       ??_C@_0DN@HHBBLAKE@JVMTI_ERROR_UNSUPPORTED_REDEFIN@ 0000000180006e30     libiterreachobj002.obj
 0002:00000e70       ??_C@_0DO@HMBGBGNA@JVMTI_ERROR_UNSUPPORTED_REDEFIN@ 0000000180006e70     libiterreachobj002.obj
 0002:00000eb0       ??_C@_0BP@PBECGKHJ@JVMTI_ERROR_UNMODIFIABLE_CLASS@ 0000000180006eb0     libiterreachobj002.obj
 0002:00000ed0       ??_C@_0BK@CANILEHF@JVMTI_ERROR_NOT_AVAILABLE@ 0000000180006ed0     libiterreachobj002.obj
 0002:00000ef0       ??_C@_0CE@INJKMEFK@JVMTI_ERROR_MUST_POSSESS_CAPABI@ 0000000180006ef0     libiterreachobj002.obj
 0002:00000f18       ??_C@_0BJ@LBFPFPDM@JVMTI_ERROR_NULL_POINTER@ 0000000180006f18     libiterreachobj002.obj
 0002:00000f38       ??_C@_0BP@CHJPNNEM@JVMTI_ERROR_ABSENT_INFORMATION@ 0000000180006f38     libiterreachobj002.obj
 0002:00000f58       ??_C@_0BP@OMFMNLC@JVMTI_ERROR_INVALID_EVENT_TYPE@ 0000000180006f58     libiterreachobj002.obj
 0002:00000f78       ??_C@_0BN@BIBNPHHO@JVMTI_ERROR_ILLEGAL_ARGUMENT@ 0000000180006f78     libiterreachobj002.obj
 0002:00000f98       ??_C@_0BK@KKNDHDCE@JVMTI_ERROR_NATIVE_METHOD@ 0000000180006f98     libiterreachobj002.obj
 0002:00000fb8       ??_C@_0BK@PMKCFHAE@JVMTI_ERROR_OUT_OF_MEMORY@ 0000000180006fb8     libiterreachobj002.obj
 0002:00000fd8       ??_C@_0BK@NNJBDMNB@JVMTI_ERROR_ACCESS_DENIED@ 0000000180006fd8     libiterreachobj002.obj
 0002:00000ff8       ??_C@_0BI@GHECLMNC@JVMTI_ERROR_WRONG_PHASE@ 0000000180006ff8     libiterreachobj002.obj
 0002:00001010       ??_C@_0BF@OLIHJOII@JVMTI_ERROR_INTERNAL@ 0000000180007010     libiterreachobj002.obj
 0002:00001028       ??_C@_0BO@EOHGKJHI@JVMTI_ERROR_UNATTACHED_THREAD@ 0000000180007028     libiterreachobj002.obj
 0002:00001048       ??_C@_0CA@LKHFDACL@JVMTI_ERROR_INVALID_ENVIRONMENT@ 0000000180007048     libiterreachobj002.obj
 0002:00001068       ??_C@_0BA@MMFHLOKK@?$DMunknown?5error?$DO@ 0000000180007068     libiterreachobj002.obj
 0002:00001078       ??_C@_0CF@CBHOKDB@throwable?5?$DN?5jni?9?$DOExceptionOccur@ 0000000180007078     libiterreachobj002.obj
 0002:000010a0       ??_C@_03OFAPEBGM@?$CFs?6@  00000001800070a0     libiterreachobj002.obj
 0002:000010a8       ??_C@_0DM@LPIGEGNJ@s?2test?2hotspot?2jtreg?2vmTestbase@ 00000001800070a8     libiterreachobj002.obj
 0002:000010e8       ??_C@_0CC@NFCNPEPK@Exception?5in?5JNI?5call?5?$CIcleared?$CJ@ 00000001800070e8     libiterreachobj002.obj
 0002:00001110       ??_C@_0BJ@IBAKFIKF@jni?9?$DOExceptionDescribe?$CI?$CJ@ 0000000180007110     libiterreachobj002.obj
 0002:00001130       ??_C@_0BG@GGKALKMH@jni?9?$DOExceptionClear?$CI?$CJ@ 0000000180007130     libiterreachobj002.obj
 0002:00001148       ??_C@_0CF@JMGFGJLJ@?$CD?5?5?5verified?5JNI?5assertion?5is?5F@ 0000000180007148     libiterreachobj002.obj
 0002:00001170       ??_C@_07KBAMPNJK@verbose@  0000000180007170     libiterreachobj002.obj
 0002:00001178       ??_C@_0DN@PKJBOLAP@nsk_jvmti_parseOptions?$CI?$CJ?3?5unexp@ 0000000180007178     libiterreachobj002.obj
 0002:000011b8       ??_C@_05IMBNNINJ@trace@    00000001800071b8     libiterreachobj002.obj
 0002:000011c0       ??_C@_0DD@BJKGNDMB@nsk_jvmti_parseOptions?$CI?$CJ?3?5no?5va@ 00000001800071c0     libiterreachobj002.obj
 0002:000011f4       ??_C@_04CGFJFPFD@none@     00000001800071f4     libiterreachobj002.obj
 0002:000011fc       ??_C@_06BMELKFMA@before@   00000001800071fc     libiterreachobj002.obj
 0002:00001204       ??_C@_05CMKPCFDK@after@    0000000180007204     libiterreachobj002.obj
 0002:0000120c       ??_C@_03NFKEKGGK@all@      000000018000720c     libiterreachobj002.obj
 0002:00001210       ??_C@_0DM@NDNJGJKE@nsk_jvmti_parseOptions?$CI?$CJ?3?5uexpe@ 0000000180007210     libiterreachobj002.obj
 0002:00001250       ??_C@_08NBBJKJO@waittime@  0000000180007250     libiterreachobj002.obj
 0002:00001260       ??_C@_0DO@CMHGAOHC@nsk_jvmti_parseOptions?$CI?$CJ?3?5not?5i@ 0000000180007260     libiterreachobj002.obj
 0002:000012a0       ??_C@_0DL@LNMPBDLN@nsk_jvmti_parseOptions?$CI?$CJ?3?5negat@ 00000001800072a0     libiterreachobj002.obj
 0002:000012e0       ??_C@_0DA@GMFJNOJH@nsk_jvmti_parseOptions?$CI?$CJ?3?5unkno@ 00000001800072e0     libiterreachobj002.obj
 0002:00001310       ??_C@_0CO@CCIAMEAN@nsk_jvmti_parseOptions?$CI?$CJ?3?5found@ 0000000180007310     libiterreachobj002.obj
 0002:00001340       ??_C@_0CJ@OEGPCGDL@nsk_jvmti_parseOptions?$CI?$CJ?3?5out?5o@ 0000000180007340     libiterreachobj002.obj
 0002:00001370       ??_C@_0DI@NMBHPGGF@nsk_jvmti_parseOptions?$CI?$CJ?3?5too?5m@ 0000000180007370     libiterreachobj002.obj
 0002:000013a8       ??_C@_03POGCGECB@?5?0?$HO@ 00000001800073a8     libiterreachobj002.obj
 0002:000013b0       ??_C@_0CB@MLNJNCLJ@?5?5jvmti?5error?3?5code?$DN?$CFd?0?5name?$DN?$CFs@ 00000001800073b0     libiterreachobj002.obj
 0002:000013d8       ??_C@_0CD@OHBGDKMK@?$CD?5?5?5jvmti?5error?3?5code?$DN?$CFd?0?5name?$DN@ 00000001800073d8     libiterreachobj002.obj
 0002:00001400       ??_C@_0CG@JNNCGPHB@?$CD?5?5?5error?5expected?3?5code?$DN?$CFd?0?5na@ 0000000180007400     libiterreachobj002.obj
 0002:00001430       ??_C@_0EB@IMGKPCGE@?$CIstr_obj?5?$DN?5jni?9?$DONewStringUTF?$CIco@ 0000000180007430     libiterreachobj002.obj
 0002:00001480       ??_C@_0EA@HFOGGBCC@s?2test?2hotspot?2jtreg?2vmTestbase@ 0000000180007480     libiterreachobj002.obj
 0002:000014c0       ??_C@_05KKCIMGE@error@     00000001800074c0     libiterreachobj002.obj
 0002:000014c8       ??_C@_0BD@HGNAOMCP@agent_data_monitor@ 00000001800074c8     libiterreachobj002.obj
 0002:000014e0       ??_C@_0EB@OGCLGKLN@javaVM?9?$DOGetEnv?$CI?$CIvoid?5?$CK?$CK?$CJ?$CGjvmti_@ 00000001800074e0     libiterreachobj002.obj
 0002:00001530       ??_C@_0EA@PNBCDMOA@s?2test?2hotspot?2jtreg?2vmTestbase@ 0000000180007530     libiterreachobj002.obj
 0002:00001570       ??_C@_0CI@DDPIFBGM@init_agent_data?$CIjvmti_env?0?5?$CGage@ 0000000180007570     libiterreachobj002.obj
 0002:00001598       ??_C@_0DI@ILAHDLMP@?$CI?$CKagentThreadProc?$CJ?$CIjvmti_env?0?5a@ 0000000180007598     libiterreachobj002.obj
 0002:000015d0       ??_C@_0BD@KDBALNLB@JVMTI?5agent?5thread@ 00000001800075d0     libiterreachobj002.obj
 0002:000015e8       ??_C@_0BB@NOKBFPFO@java?1lang?1Thread@ 00000001800075e8     libiterreachobj002.obj
 0002:000015fc       ??_C@_06FALKBLGB@?$DMinit?$DO@ 00000001800075fc     libiterreachobj002.obj
 0002:00001608       ??_C@_0BG@IKDDPPGD@?$CILjava?1lang?1String?$DL?$CJV@ 0000000180007608     libiterreachobj002.obj
 0002:00001620       ??_C@_0EB@IFJBFEKC@?$CIthreadClass?5?$DN?5jni_env?9?$DOFindCla@ 0000000180007620     libiterreachobj002.obj
 0002:00001670       ??_C@_0GF@FGFIBKKL@?$CIthreadCtor?5?$DN?5jni_env?9?$DOGetMetho@ 0000000180007670     libiterreachobj002.obj
 0002:000016d8       ??_C@_0DN@NCPDJLOG@?$CIthreadName?5?$DN?5jni_env?9?$DONewStrin@ 00000001800076d8     libiterreachobj002.obj
 0002:00001720       ??_C@_0FE@PFKODBGC@?$CIthreadObject?5?$DN?5jni_env?9?$DONewObj@ 0000000180007720     libiterreachobj002.obj
 0002:00001780       ??_C@_0ED@HOBAHHJI@?$CIthreadGlobalRef?5?$DN?5jni_env?9?$DONew@ 0000000180007780     libiterreachobj002.obj
 0002:000017d0       ??_C@_0FN@HNJJAHFC@jvmti_env?9?$DORunAgentThread?$CIagent@ 00000001800077d0     libiterreachobj002.obj
 0002:00001830       ??_C@_0EA@MOJDNKDF@Debuggee?5status?5sync?5aborted?5be@ 0000000180007830     libiterreachobj002.obj
 0002:00001870       ??_C@_0CO@PGPGMHBJ@No?5status?5sync?5occured?5for?5time@ 0000000180007870     libiterreachobj002.obj
 0002:000018a0       ??_C@_0CL@DOEBDPKJ@Debuggee?5was?5not?5suspended?5on?5s@ 00000001800078a0     libiterreachobj002.obj
 0002:000018d0       ??_C@_0EA@EEOEJAEN@status?5?$DN?5syncDebuggeeStatus?$CIjni@ 00000001800078d0     libiterreachobj002.obj
 0002:00001910       ??_C@_0BL@JBCFNBMB@nsk_jvmti_resetAgentData?$CI?$CJ@ 0000000180007910     libiterreachobj002.obj
 0002:00001930       ??_C@_0EL@LPBEELIP@s?2test?2hotspot?2jtreg?2vmTestbase@ 0000000180007930     libiterreachobj002.obj
 0002:00001980       ??_C@_0CK@JDAMFDMJ@jvmti?9?$DOSetTag?$CIo?0?5tag?$CJ?5?$DN?$DN?5JVMTI_@ 0000000180007980     libiterreachobj002.obj
 0002:000019b0       ??_C@_0CC@DAMNHKNI@Can?8t?5set?5tag?5?$CFli?5for?5object?5?$CFl@ 00000001800079b0     libiterreachobj002.obj
 0002:000019d8       ??_C@_0DL@HAJPNKEF@jvmti?9?$DOGetObjectHashCode?$CIo?0?5?$CGha@ 00000001800079d8     libiterreachobj002.obj
 0002:00001a18       ??_C@_0BL@JFPIEOBF@Can?8t?5get?5hash?5object?5?$CFlx?6@ 0000000180007a18     libiterreachobj002.obj
 0002:00001a38       ??_C@_0BG@DICPHBKN@setTag?3?5?$CF08x?5?$DM?9?5?$CF?53li@ 0000000180007a38     libiterreachobj002.obj
 0002:00001a50       ??_C@_0DH@FCEEBDMJ@?$CIs?5?$DN?5jni?9?$DOGetStringUTFChars?$CIsIn@ 0000000180007a50     libiterreachobj002.obj
 0002:00001a88       ??_C@_0BJ@OKKGHDCN@Can?8t?5get?5string?5at?5?$CF?$CDp?6@ 0000000180007a88     libiterreachobj002.obj
 0002:00001aa8       ??_C@_0BP@EKFLGGFJ@Can?8t?5get?5string?5at?5?$CF?$CDp?3?5null?6@ 0000000180007aa8     libiterreachobj002.obj
 0002:00001ac8       ??_C@_06ICODBHCL@?5?1?1?5?$CFs@ 0000000180007ac8     libiterreachobj002.obj
 0002:00001ad0       ??_C@_0DB@KGFPLEGO@?$CIr?5?$DN?5jvmti?9?$DOGetTag?$CIo?0?5?$CGtag?$CJ?$CJ?5?$DN?$DN@ 0000000180007ad0     libiterreachobj002.obj
 0002:00001b08       ??_C@_0CO@PDAGBCGJ@Can?8t?5GetTag?5for?5object?5?$CFlx?4?5Re@ 0000000180007b08     libiterreachobj002.obj
 0002:00001b38       ??_C@_0CH@HPEODOHC@TEST_BUG?3?5Max?4?5number?5of?5refs?5r@ 0000000180007b38     libiterreachobj002.obj
 0002:00001b60       ??_C@_0DI@PHFCABIM@?$CIr?5?$DN?5jvmti?9?$DOGetTag?$CIfrom?0?5?$CGtagFr@ 0000000180007b60     libiterreachobj002.obj
 0002:00001b98       ??_C@_0DI@MDEGFNKD@TEST_BUG?3?5Can?8t?5GetTag?5for?5obje@ 0000000180007b98     libiterreachobj002.obj
 0002:00001bd0       ??_C@_0DE@MLELJAHM@?$CIr?5?$DN?5jvmti?9?$DOGetTag?$CIto?0?5?$CGtagTo?$CJ?$CJ@ 0000000180007bd0     libiterreachobj002.obj
 0002:00001c10       ??_C@_0EH@LGFKMLEF@jvmti?9?$DOAllocate?$CI?$CIsizeof?$CIObjectD@ 0000000180007c10     libiterreachobj002.obj
 0002:00001c60       ??_C@_0GK@PHOODIBM@s?2test?2hotspot?2jtreg?2vmTestbase@ 0000000180007c60     libiterreachobj002.obj
 0002:00001cd0       ??_C@_0FB@CLHKKOJM@heapRootCallbackForFirstObjects@ 0000000180007cd0     libiterreachobj002.obj
 0002:00001d30       ??_C@_0EJ@DGEBBCHI@heapRootCallbackForSecondObject@ 0000000180007d30     libiterreachobj002.obj
 0002:00001d80       ??_C@_0DG@PPFKFGPA@jvmti?9?$DODeallocate?$CI?$CIunsigned?5cha@ 0000000180007d80     libiterreachobj002.obj
 0002:00001dc0       ??_C@_0FE@OOJLJBIK@heapRootCallbackForSecondObject@ 0000000180007dc0     libiterreachobj002.obj
 0002:00001e20       ??_C@_0FH@ODACJBMA@stackReferenceCallbackForFirstO@ 0000000180007e20     libiterreachobj002.obj
 0002:00001e80       ??_C@_0EP@OOIOCEJH@stackReferenceCallbackForSecond@ 0000000180007e80     libiterreachobj002.obj
 0002:00001ed0       ??_C@_0FK@INDNJFKE@stackReferenceCallbackForSecond@ 0000000180007ed0     libiterreachobj002.obj
 0002:00001f30       ??_C@_0FI@BMPNAMJC@objectReferenceCallbackForFirst@ 0000000180007f30     libiterreachobj002.obj
 0002:00001f90       ??_C@_0FA@GHLPJKAP@objectReferenceCallbackForSecon@ 0000000180007f90     libiterreachobj002.obj
 0002:00001fe0       ??_C@_0FL@LOIHEFP@objectReferenceCallbackForSecon@ 0000000180007fe0     libiterreachobj002.obj
 0002:00002040       ??_C@_0BI@BGHFFELJ@Wait?5for?5debugee?5start?6@ 0000000180008040     libiterreachobj002.obj
 0002:00002058       ??_C@_0BP@LAIJOMPC@nsk_jvmti_waitForSync?$CItimeout?$CJ@ 0000000180008058     libiterreachobj002.obj
 0002:00002080       ??_C@_0EI@FKJPPDKE@Calling?5IterateOverReachableObj@ 0000000180008080     libiterreachobj002.obj
 0002:000020d0       ??_C@_0LK@MMKADNDN@jvmti?9?$DOIterateOverReachableObje@ 00000001800080d0     libiterreachobj002.obj
 0002:00002190       ??_C@_0ED@GPIPIMCM@First?5IterateOverReachableObjec@ 0000000180008190     libiterreachobj002.obj
 0002:000021e0       ??_C@_0EF@JMNKCFDI@Number?5of?5objects?5the?5first?5Ite@ 00000001800081e0     libiterreachobj002.obj
 0002:00002228       ??_C@_0DC@DFJJAFOM@jvmti?9?$DODeallocate?$CI?$CIunsigned?5cha@ 0000000180008228     libiterreachobj002.obj
 0002:00002260       ??_C@_0DE@OFCOFDAK@Unable?5to?5deallocate?5last?5unnec@ 0000000180008260     libiterreachobj002.obj
 0002:000022a0       ??_C@_0FG@FHPMDIE@jvmti?9?$DOAllocate?$CI?$CIobjectCount?5?$CK?5@ 00000001800082a0     libiterreachobj002.obj
 0002:00002300       ??_C@_0FJ@OEBOHECC@jvmti?9?$DOAllocate?$CI?$CIobjectCountMax@ 0000000180008300     libiterreachobj002.obj
 0002:00002360       ??_C@_0EK@LFEMOEO@Calling?5IterateOverReachableObj@ 0000000180008360     libiterreachobj002.obj
 0002:000023b0       ??_C@_0LN@LKHAGOCM@jvmti?9?$DOIterateOverReachableObje@ 00000001800083b0     libiterreachobj002.obj
 0002:00002470       ??_C@_0IC@NKDKBODJ@Deallocate?5func?4?5hasn?8t?5been?5ca@ 0000000180008470     libiterreachobj002.obj
 0002:000024f8       ??_C@_0CO@GLOLACHK@Unable?5to?5deallocate?5descriptor@ 00000001800084f8     libiterreachobj002.obj
 0002:00002528       ??_C@_0DB@BPEANDEF@jvmti?9?$DODeallocate?$CI?$CIunsigned?5cha@ 0000000180008528     libiterreachobj002.obj
 0002:00002560       ??_C@_0DH@GODCMBGD@jvmti?9?$DODeallocate?$CI?$CIunsigned?5cha@ 0000000180008560     libiterreachobj002.obj
 0002:00002598       ??_C@_0BH@HPEOJMHL@Let?5debugee?5to?5finish?6@ 0000000180008598     libiterreachobj002.obj
 0002:000025b0       ??_C@_0BH@LECMGIIA@nsk_jvmti_resumeSync?$CI?$CJ@ 00000001800085b0     libiterreachobj002.obj
 0002:000025c8       ??_C@_0CA@MNKGCBCG@nsk_jvmti_parseOptions?$CIoptions?$CJ@ 00000001800085c8     libiterreachobj002.obj
 0002:000025e8       ??_C@_0DN@MIAMNFPH@?$CIjvmti?5?$DN?5nsk_jvmti_createJVMTIE@ 00000001800085e8     libiterreachobj002.obj
 0002:00002628       ??_C@_0BO@DBKDIPGD@jvmti?9?$DOAddCapabilities?$CI?$CGcaps?$CJ@ 0000000180008628     libiterreachobj002.obj
 0002:00002648       ??_C@_0BO@IAKFILDF@jvmti?9?$DOGetCapabilities?$CI?$CGcaps?$CJ@ 0000000180008648     libiterreachobj002.obj
 0002:00002668       ??_C@_0CL@NEGLJNIP@Warning?3?5tagging?5objects?5is?5not@ 0000000180008668     libiterreachobj002.obj
 0002:00002698       ??_C@_0DM@HHPBGDMK@Warning?3?5generation?5of?5object?5f@ 0000000180008698     libiterreachobj002.obj
 0002:000026d8       ??_C@_0BN@HGIKGGD@setting?5event?5callbacks?5?4?4?4?6@ 00000001800086d8     libiterreachobj002.obj
 0002:000026f8       ??_C@_0DI@NJCFGEGC@jvmti?9?$DOSetEventCallbacks?$CI?$CGcallb@ 00000001800086f8     libiterreachobj002.obj
 0002:00002730       ??_C@_0BP@KGJAPGFD@setting?5event?5callbacks?5done?4?6@ 0000000180008730     libiterreachobj002.obj
 0002:00002750       ??_C@_0BL@PCGFMOMJ@enabling?5JVMTI?5events?5?4?4?4?6@ 0000000180008750     libiterreachobj002.obj
 0002:00002770       ??_C@_0FA@KLKMFDPK@jvmti?9?$DOSetEventNotificationMode@ 0000000180008770     libiterreachobj002.obj
 0002:000027c0       ??_C@_0BL@FOKCDLBD@enabling?5the?5events?5done?4?6@ 00000001800087c0     libiterreachobj002.obj
 0002:000027e0       ??_C@_0CL@PIACJIPK@nsk_jvmti_setAgentProc?$CIagentPro@ 00000001800087e0     libiterreachobj002.obj
 0002:00002820       ??_C@_1EC@JIJBPKFM@?$AAa?$AAp?$AAi?$AA?9?$AAm?$AAs?$AA?9?$AAw?$AAi?$AAn?$AA?9?$AAc?$AAo?$AAr?$AAe@ 0000000180008820     MSVCRT:thread_safe_statics.obj
 0002:00002868       ??_C@_1BK@MGMFAEKH@?$AAk?$AAe?$AAr?$AAn?$AAe?$AAl?$AA3?$AA2?$AA?4?$AAd?$AAl?$AAl@ 0000000180008868     MSVCRT:thread_safe_statics.obj
 0002:00002888       ??_C@_0BJ@JEBJOJFJ@SleepConditionVariableCS@ 0000000180008888     MSVCRT:thread_safe_statics.obj
 0002:000028a8       ??_C@_0BJ@PGPPEPCC@WakeAllConditionVariable@ 00000001800088a8     MSVCRT:thread_safe_statics.obj
 0002:000028c8       _pDefaultRawDllMain        00000001800088c8     MSVCRT:dll_dllmain.obj
 0002:000028c8       _pRawDllMain               00000001800088c8     MSVCRT:dll_dllmain.obj
 0002:000028d0       __xmm@ffffffffffffffffffffffffffffffff 00000001800088d0     MSVCRT:utility.obj
 0002:000028e0       _load_config_used          00000001800088e0     MSVCRT:loadcfg.obj
 0002:00002b00       _tls_used                  0000000180008b00     MSVCRT:tlssup.obj
 0002:00002b28       __volatile_metadata        0000000180008b28     <linker-defined>
 0002:00002fd0       __rtc_iaa                  0000000180008fd0     MSVCRT:initsect.obj
 0002:00002fd8       __rtc_izz                  0000000180008fd8     MSVCRT:initsect.obj
 0002:00002fe0       __rtc_taa                  0000000180008fe0     MSVCRT:initsect.obj
 0002:00002fe8       __rtc_tzz                  0000000180008fe8     MSVCRT:initsect.obj
 0002:00002ff0       _tls_start                 0000000180008ff0     MSVCRT:tlssup.obj
 0002:00002ff4       _Init_thread_epoch         0000000180008ff4     MSVCRT:thread_safe_statics.obj
 0002:00002ff8       _tls_end                   0000000180008ff8     MSVCRT:tlssup.obj
 0002:00003698       __IMPORT_DESCRIPTOR_KERNEL32 0000000180009698     kernel32:KERNEL32.dll
 0002:000036ac       __IMPORT_DESCRIPTOR_VCRUNTIME140 00000001800096ac     vcruntime:VCRUNTIME140.dll
 0002:000036c0       __IMPORT_DESCRIPTOR_api-ms-win-crt-heap-l1-1-0 00000001800096c0     ucrt:api-ms-win-crt-heap-l1-1-0.dll
 0002:000036d4       __IMPORT_DESCRIPTOR_api-ms-win-crt-runtime-l1-1-0 00000001800096d4     ucrt:api-ms-win-crt-runtime-l1-1-0.dll
 0002:000036e8       __IMPORT_DESCRIPTOR_api-ms-win-crt-convert-l1-1-0 00000001800096e8     ucrt:api-ms-win-crt-convert-l1-1-0.dll
 0002:000036fc       __IMPORT_DESCRIPTOR_api-ms-win-crt-stdio-l1-1-0 00000001800096fc     ucrt:api-ms-win-crt-stdio-l1-1-0.dll
 0002:00003710       __IMPORT_DESCRIPTOR_api-ms-win-crt-string-l1-1-0 0000000180009710     ucrt:api-ms-win-crt-string-l1-1-0.dll
 0002:00003724       __NULL_IMPORT_DESCRIPTOR   0000000180009724     kernel32:KERNEL32.dll
 0003:00000030       _Init_global_epoch         000000018000a030     MSVCRT:thread_safe_statics.obj
 0003:00000040       __security_cookie          000000018000a040     MSVCRT:gs_cookie.obj
 0003:00000048       __security_cookie_complement 000000018000a048     MSVCRT:gs_cookie.obj
 0003:00000050       __scrt_native_dllmain_reason 000000018000a050     MSVCRT:utility.obj
 0003:00000058       __isa_available            000000018000a058     MSVCRT:cpu_disp.obj
 0003:0000005c       __isa_enabled              000000018000a05c     MSVCRT:cpu_disp.obj
 0003:00000060       __memset_fast_string_threshold 000000018000a060     MSVCRT:cpu_disp.obj
 0003:00000068       __memset_nt_threshold      000000018000a068     MSVCRT:cpu_disp.obj
 0003:00000070       __scrt_ucrt_dll_is_in_use  000000018000a070     MSVCRT:ucrt_stubs.obj
 0003:00000080       g_wrongHeapCallbacks       000000018000a080     libiterreachobj002.obj
 0003:00000100       g_szTagInfo                000000018000a100     libiterreachobj002.obj
 0003:00002040       g_tagFlags                 000000018000c040     libiterreachobj002.obj
 0003:00002428       g_refsToVerifyCnt          000000018000c428     libiterreachobj002.obj
 0003:0000242c       g_fakeUserData             000000018000c42c     libiterreachobj002.obj
 0003:00002430       g_tagVisitCount            000000018000c430     libiterreachobj002.obj
 0003:000033d0       g_refsToVerify             000000018000d3d0     libiterreachobj002.obj
 0003:0001aad0       g_userDataError            0000000180024ad0     libiterreachobj002.obj
 0003:0001adf8       ?_OptionsStorage@?1??__local_stdio_printf_options@@9@4_KA 0000000180024df8     libiterreachobj002.obj
 0003:0001b3b8       _tls_index                 00000001800253b8     MSVCRT:tlssup.obj
 0003:0001b3c0       __scrt_current_native_startup_state 00000001800253c0     MSVCRT:utility.obj
 0003:0001b3c8       __scrt_native_startup_lock 00000001800253c8     MSVCRT:utility.obj
 0003:0001b408       __scrt_debugger_hook_flag  0000000180025408     MSVCRT:utility_desktop.obj
 0003:0001b410       ?__type_info_root_node@@3U__type_info_node@@A 0000000180025410     MSVCRT:tncleanup.obj
 0003:0001b420       ?_OptionsStorage@?1??__local_stdio_scanf_options@@9@4_KA 0000000180025420     MSVCRT:default_local_stdio_options.obj
 0003:0001b428       __favor                    0000000180025428     MSVCRT:cpu_disp.obj
 0003:0001b430       __dyn_tls_init_callback    0000000180025430     <common>

 entry point at        0001:00003850

 Static symbols

 0000:fffd8000       .debug$S                   0000000180000000     iterreachobj002.exp
 0000:fffd8000       .debug$S                   0000000180000000     vcruntime:VCRUNTIME140.dll
 0000:fffd8000       .debug$S                   0000000180000000     vcruntime:VCRUNTIME140.dll
 0000:fffd8000       .debug$S                   0000000180000000     vcruntime:VCRUNTIME140.dll
 0000:fffd8000       .debug$S                   0000000180000000     vcruntime:VCRUNTIME140.dll
 0000:fffd8000       .debug$S                   0000000180000000     vcruntime:VCRUNTIME140.dll
 0000:fffd8000       .debug$S                   0000000180000000     vcruntime:VCRUNTIME140.dll
 0000:fffd8000       .debug$S                   0000000180000000     vcruntime:VCRUNTIME140.dll
 0000:fffd8000       .debug$S                   0000000180000000     ucrt:api-ms-win-crt-convert-l1-1-0.dll
 0000:fffd8000       .debug$S                   0000000180000000     ucrt:api-ms-win-crt-heap-l1-1-0.dll
 0000:fffd8000       .debug$S                   0000000180000000     ucrt:api-ms-win-crt-heap-l1-1-0.dll
 0000:fffd8000       .debug$S                   0000000180000000     ucrt:api-ms-win-crt-heap-l1-1-0.dll
 0000:fffd8000       .debug$S                   0000000180000000     ucrt:api-ms-win-crt-heap-l1-1-0.dll
 0000:fffd8000       .debug$S                   0000000180000000     ucrt:api-ms-win-crt-runtime-l1-1-0.dll
 0000:fffd8000       .debug$S                   0000000180000000     ucrt:api-ms-win-crt-runtime-l1-1-0.dll
 0000:fffd8000       .debug$S                   0000000180000000     ucrt:api-ms-win-crt-runtime-l1-1-0.dll
 0000:fffd8000       .debug$S                   0000000180000000     ucrt:api-ms-win-crt-runtime-l1-1-0.dll
 0000:fffd8000       .debug$S                   0000000180000000     ucrt:api-ms-win-crt-runtime-l1-1-0.dll
 0000:fffd8000       .debug$S                   0000000180000000     ucrt:api-ms-win-crt-runtime-l1-1-0.dll
 0000:fffd8000       .debug$S                   0000000180000000     ucrt:api-ms-win-crt-runtime-l1-1-0.dll
 0000:fffd8000       .debug$S                   0000000180000000     ucrt:api-ms-win-crt-runtime-l1-1-0.dll
 0000:fffd8000       .debug$S                   0000000180000000     ucrt:api-ms-win-crt-runtime-l1-1-0.dll
 0000:fffd8000       .debug$S                   0000000180000000     ucrt:api-ms-win-crt-runtime-l1-1-0.dll
 0000:fffd8000       .debug$S                   0000000180000000     ucrt:api-ms-win-crt-runtime-l1-1-0.dll
 0000:fffd8000       .debug$S                   0000000180000000     ucrt:api-ms-win-crt-runtime-l1-1-0.dll
 0000:fffd8000       .debug$S                   0000000180000000     ucrt:api-ms-win-crt-runtime-l1-1-0.dll
 0000:fffd8000       .debug$S                   0000000180000000     ucrt:api-ms-win-crt-runtime-l1-1-0.dll
 0000:fffd8000       .debug$S                   0000000180000000     ucrt:api-ms-win-crt-runtime-l1-1-0.dll
 0000:fffd8000       .debug$S                   0000000180000000     ucrt:api-ms-win-crt-runtime-l1-1-0.dll
 0000:fffd8000       .debug$S                   0000000180000000     ucrt:api-ms-win-crt-stdio-l1-1-0.dll
 0000:fffd8000       .debug$S                   0000000180000000     ucrt:api-ms-win-crt-stdio-l1-1-0.dll
 0000:fffd8000       .debug$S                   0000000180000000     ucrt:api-ms-win-crt-stdio-l1-1-0.dll
 0000:fffd8000       .debug$S                   0000000180000000     ucrt:api-ms-win-crt-stdio-l1-1-0.dll
 0000:fffd8000       .debug$S                   0000000180000000     ucrt:api-ms-win-crt-stdio-l1-1-0.dll
 0000:fffd8000       .debug$S                   0000000180000000     ucrt:api-ms-win-crt-stdio-l1-1-0.dll
 0000:fffd8000       .debug$S                   0000000180000000     ucrt:api-ms-win-crt-stdio-l1-1-0.dll
 0000:fffd8000       .debug$S                   0000000180000000     ucrt:api-ms-win-crt-stdio-l1-1-0.dll
 0000:fffd8000       .debug$S                   0000000180000000     ucrt:api-ms-win-crt-stdio-l1-1-0.dll
 0000:fffd8000       .debug$S                   0000000180000000     ucrt:api-ms-win-crt-stdio-l1-1-0.dll
 0000:fffd8000       .debug$S                   0000000180000000     ucrt:api-ms-win-crt-string-l1-1-0.dll
 0000:fffd8000       .debug$S                   0000000180000000     ucrt:api-ms-win-crt-string-l1-1-0.dll
 0000:fffd8000       .debug$S                   0000000180000000     ucrt:api-ms-win-crt-string-l1-1-0.dll
 0000:fffd8000       .debug$S                   0000000180000000     ucrt:api-ms-win-crt-string-l1-1-0.dll
 0000:fffd8000       .debug$S                   0000000180000000     ucrt:api-ms-win-crt-string-l1-1-0.dll
 0000:fffd8000       .debug$S                   0000000180000000     ucrt:api-ms-win-crt-string-l1-1-0.dll
 0000:fffd8000       .debug$S                   0000000180000000     ucrt:api-ms-win-crt-string-l1-1-0.dll
 0000:fffd8000       .debug$S                   0000000180000000     ucrt:api-ms-win-crt-string-l1-1-0.dll
 0000:fffd8000       .debug$S                   0000000180000000     kernel32:KERNEL32.dll
 0000:fffd8000       .debug$S                   0000000180000000     kernel32:KERNEL32.dll
 0000:fffd8000       .debug$S                   0000000180000000     kernel32:KERNEL32.dll
 0000:fffd8000       .debug$S                   0000000180000000     kernel32:KERNEL32.dll
 0000:fffd8000       .debug$S                   0000000180000000     kernel32:KERNEL32.dll
 0000:fffd8000       .debug$S                   0000000180000000     kernel32:KERNEL32.dll
 0000:fffd8000       .debug$S                   0000000180000000     kernel32:KERNEL32.dll
 0000:fffd8000       .debug$S                   0000000180000000     kernel32:KERNEL32.dll
 0000:fffd8000       .debug$S                   0000000180000000     kernel32:KERNEL32.dll
 0000:fffd8000       .debug$S                   0000000180000000     kernel32:KERNEL32.dll
 0000:fffd8000       .debug$S                   0000000180000000     kernel32:KERNEL32.dll
 0000:fffd8000       .debug$S                   0000000180000000     kernel32:KERNEL32.dll
 0000:fffd8000       .debug$S                   0000000180000000     kernel32:KERNEL32.dll
 0000:fffd8000       .debug$S                   0000000180000000     kernel32:KERNEL32.dll
 0000:fffd8000       .debug$S                   0000000180000000     kernel32:KERNEL32.dll
 0000:fffd8000       .debug$S                   0000000180000000     kernel32:KERNEL32.dll
 0000:fffd8000       .debug$S                   0000000180000000     kernel32:KERNEL32.dll
 0000:fffd8000       .debug$S                   0000000180000000     kernel32:KERNEL32.dll
 0000:fffd8000       .debug$S                   0000000180000000     kernel32:KERNEL32.dll
 0000:fffd8000       .debug$S                   0000000180000000     kernel32:KERNEL32.dll
 0000:fffd8000       .debug$S                   0000000180000000     kernel32:KERNEL32.dll
 0000:fffd8000       .debug$S                   0000000180000000     kernel32:KERNEL32.dll
 0000:fffd8000       .debug$S                   0000000180000000     kernel32:KERNEL32.dll
 0000:fffd8000       .debug$S                   0000000180000000     kernel32:KERNEL32.dll
 0000:fffd8000       .debug$S                   0000000180000000     kernel32:KERNEL32.dll
 0000:fffd8000       .debug$S                   0000000180000000     kernel32:KERNEL32.dll
 0000:fffd8000       .debug$S                   0000000180000000     kernel32:KERNEL32.dll
 0000:fffd8000       .debug$S                   0000000180000000     kernel32:KERNEL32.dll
 0001:00000ffc       addRefToVerify             0000000180001ffc f   libiterreachobj002.obj
 0001:00001070       agentProc                  0000000180002070 f   libiterreachobj002.obj
 0001:000016bc       agentThreadWrapper         00000001800026bc f   libiterreachobj002.obj
 0001:00001810       check_option               0000000180002810 f   libiterreachobj002.obj
 0001:00001a58       file_basename              0000000180002a58 f   libiterreachobj002.obj
 0001:00002d5c       startAgentThreadWrapper    0000000180003d5c f   libiterreachobj002.obj
 0001:00003088       syncDebuggeeStatus         0000000180004088 f   libiterreachobj002.obj
 0001:00003310       capture_previous_context   0000000180004310 f   MSVCRT:gs_report.obj
 0001:00003384       ?__scrt_initialize_thread_safe_statics@@YAHXZ 0000000180004384 f   MSVCRT:thread_safe_statics.obj
 0001:00003454       ?__scrt_uninitialize_thread_safe_statics@@YAXXZ 0000000180004454 f   MSVCRT:thread_safe_statics.obj
 0001:00003500       $$000000                   0000000180004500     MSVCRT:amdsecgs.obj
 0001:00003530       ?dllmain_crt_dispatch@@YAHQEAUHINSTANCE__@@KQEAX@Z 0000000180004530 f   MSVCRT:dll_dllmain.obj
 0001:00003580       ?dllmain_crt_process_attach@@YAHQEAUHINSTANCE__@@QEAX@Z 0000000180004580 f   MSVCRT:dll_dllmain.obj
 0001:00003698       ?dllmain_crt_process_detach@@YAH_N@Z 0000000180004698 f   MSVCRT:dll_dllmain.obj
 0001:0000371c       ?dllmain_dispatch@@YAHQEAUHINSTANCE__@@KQEAX@Z 000000018000471c f   MSVCRT:dll_dllmain.obj
 0001:00004130       $$000000                   0000000180005130     MSVCRT:guard_dispatch.obj
 0001:00004150       $$000000                   0000000180005150     MSVCRT:guard_xfg_dispatch.obj
 0001:00004166       ?fin$0@?0??dllmain_crt_process_attach@@YAHQEAUHINSTANCE__@@QEAX@Z@4HA 0000000180005166 f   MSVCRT:dll_dllmain.obj
 0001:0000417d       ?fin$0@?0??dllmain_crt_process_detach@@YAH_N@Z@4HA 000000018000517d f   MSVCRT:dll_dllmain.obj
 0001:00004196       ?fin$1@?0??dllmain_crt_process_detach@@YAH_N@Z@4HA 0000000180005196 f   MSVCRT:dll_dllmain.obj
 0001:000041aa       ?filt$0@?0??dllmain_dispatch@@YAHQEAUHINSTANCE__@@KQEAX@Z@4HA 00000001800051aa f   MSVCRT:dll_dllmain.obj
 0001:000041e0       __scrt_is_nonwritable_in_current_image$filt$0 00000001800051e0 f   MSVCRT:utility.obj
 0002:00000218       ?__scrt_initialize_tss_var@@3P6AHXZEA 0000000180006218     MSVCRT:thread_safe_statics.obj
 0002:00000340       ?opcLengths@@3QBEB         0000000180006340     libiterreachobj002.obj
 0002:00002810       GS_ExceptionPointers       0000000180008810     MSVCRT:gs_report.obj
 0002:00003000       $unwind$fprintf            0000000180009000     libiterreachobj002.obj
 0002:0000300c       $unwind$printf             000000018000900c     libiterreachobj002.obj
 0002:00003018       $unwind$?NewObject@JNIEnv_@@QEAAPEAV_jobject@@PEAV_jclass@@PEAU_jmethodID@@ZZ 0000000180009018     libiterreachobj002.obj
 0002:00003018       $unwind$nsk_lcomplain      0000000180009018     libiterreachobj002.obj
 0002:00003018       $unwind$nsk_ldisplay       0000000180009018     libiterreachobj002.obj
 0002:00003020       $unwind$nsk_lvdisplay      0000000180009020     libiterreachobj002.obj
 0002:00003020       $unwind$_RTC_Initialize    0000000180009020     MSVCRT:initsect.obj
 0002:00003020       $unwind$_RTC_Terminate     0000000180009020     MSVCRT:initsect.obj
 0002:00003020       $unwind$?__scrt_initialize_thread_safe_statics@@YAHXZ 0000000180009020     MSVCRT:thread_safe_statics.obj
 0002:0000302c       $unwind$nsk_complain       000000018000902c     libiterreachobj002.obj
 0002:0000302c       $unwind$nsk_printf         000000018000902c     libiterreachobj002.obj
 0002:00003034       $unwind$nsk_lvcomplain     0000000180009034     libiterreachobj002.obj
 0002:0000304c       $unwind$nsk_ltrace         000000018000904c     libiterreachobj002.obj
 0002:0000304c       $unwind$__report_gsfailure 000000018000904c     MSVCRT:gs_report.obj
 0002:00003054       $unwind$nsk_lvtrace        0000000180009054     libiterreachobj002.obj
 0002:00003054       $unwind$__raise_securityfailure 0000000180009054     MSVCRT:gs_report.obj
 0002:00003054       $unwind$__scrt_initialize_crt 0000000180009054     MSVCRT:utility.obj
 0002:00003054       $unwind$__scrt_initialize_onexit_tables 0000000180009054     MSVCRT:utility.obj
 0002:00003054       $unwind$__scrt_release_startup_lock 0000000180009054     MSVCRT:utility.obj
 0002:00003054       $unwind$__scrt_uninitialize_crt 0000000180009054     MSVCRT:utility.obj
 0002:00003054       $unwind$_onexit            0000000180009054     MSVCRT:utility.obj
 0002:0000305c       $unwind$nsk_lverify        000000018000905c     libiterreachobj002.obj
 0002:0000306c       $unwind$nsk_vprintf        000000018000906c     libiterreachobj002.obj
 0002:0000307c       $unwind$?nsk_jni_lverify@@YAHHPEAUJNIEnv_@@HQEBDH1ZZ 000000018000907c     libiterreachobj002.obj
 0002:00003090       $unwind$?nsk_jni_check_exception@@YAHPEAUJNIEnv_@@QEBDH@Z 0000000180009090     libiterreachobj002.obj
 0002:000030ac       $unwind$nsk_jvmti_parseOptions 00000001800090ac     libiterreachobj002.obj
 0002:000030c8       $unwind$nsk_jvmti_createJVMTIEnv 00000001800090c8     libiterreachobj002.obj
 0002:000030dc       $unwind$check_option       00000001800090dc     libiterreachobj002.obj
 0002:000030dc       $unwind$nsk_jvmti_waitForSync 00000001800090dc     libiterreachobj002.obj
 0002:000030dc       $unwind$_DllMainCRTStartup 00000001800090dc     MSVCRT:dll_dllmain.obj
 0002:000030ec       $unwind$Java_nsk_jvmti_unit_FollowReferences_FollowRefObjects_resetTags 00000001800090ec     libiterreachobj002.obj
 0002:000030ec       $unwind$addRefToVerify     00000001800090ec     libiterreachobj002.obj
 0002:000030ec       $unwind$nsk_jvmti_resetAgentData 00000001800090ec     libiterreachobj002.obj
 0002:000030ec       $unwind$nsk_jvmti_resumeSync 00000001800090ec     libiterreachobj002.obj
 0002:000030ec       $unwind$__scrt_initialize_default_local_stdio_options 00000001800090ec     MSVCRT:default_local_stdio_options.obj
 0002:000030ec       $unwind$?dllmain_crt_dispatch@@YAHQEAUHINSTANCE__@@KQEAX@Z 00000001800090ec     MSVCRT:dll_dllmain.obj
 0002:000030ec       $unwind$DllMain            00000001800090ec     MSVCRT:dll_dllmain_stub.obj
 0002:000030ec       $unwind$__GSHandlerCheck   00000001800090ec     MSVCRT:gshandler.obj
 0002:000030ec       $unwind$?__scrt_uninitialize_thread_safe_statics@@YAXXZ 00000001800090ec     MSVCRT:thread_safe_statics.obj
 0002:000030ec       $unwind$__scrt_acquire_startup_lock 00000001800090ec     MSVCRT:utility.obj
 0002:000030ec       $unwind$__scrt_dllmain_after_initialize_c 00000001800090ec     MSVCRT:utility.obj
 0002:000030ec       $unwind$__scrt_dllmain_before_initialize_c 00000001800090ec     MSVCRT:utility.obj
 0002:000030ec       $unwind$__scrt_dllmain_crt_thread_attach 00000001800090ec     MSVCRT:utility.obj
 0002:000030ec       $unwind$__scrt_dllmain_crt_thread_detach 00000001800090ec     MSVCRT:utility.obj
 0002:000030ec       $unwind$__scrt_dllmain_uninitialize_c 00000001800090ec     MSVCRT:utility.obj
 0002:000030ec       $unwind$__scrt_dllmain_uninitialize_critical 00000001800090ec     MSVCRT:utility.obj
 0002:000030ec       $unwind$atexit             00000001800090ec     MSVCRT:utility.obj
 0002:000030f4       $unwind$nsk_jvmti_lverify  00000001800090f4     libiterreachobj002.obj
 0002:00003108       $unwind$exitOnError        0000000180009108     libiterreachobj002.obj
 0002:00003118       $unwind$Java_nsk_share_jvmti_ArgumentHandler_getAgentOptionsString 0000000180009118     libiterreachobj002.obj
 0002:0000312c       $unwind$Java_nsk_jvmti_unit_FollowReferences_FollowRefObjects_getTag 000000018000912c     libiterreachobj002.obj
 0002:0000312c       $unwind$Java_nsk_share_jvmti_DebugeeClass_checkStatus 000000018000912c     libiterreachobj002.obj
 0002:0000312c       $unwind$agentThreadWrapper 000000018000912c     libiterreachobj002.obj
 0002:0000313c       $unwind$Agent_Initialize   000000018000913c     libiterreachobj002.obj
 0002:0000313c       $unwind$agentProc          000000018000913c     libiterreachobj002.obj
 0002:0000313c       $unwind$startAgentThreadWrapper 000000018000913c     libiterreachobj002.obj
 0002:00003158       $unwind$syncDebuggeeStatus 0000000180009158     libiterreachobj002.obj
 0002:00003158       $unwind$__scrt_dllmain_exception_filter 0000000180009158     MSVCRT:utility.obj
 0002:0000316c       $unwind$Java_nsk_share_jvmti_DebugeeClass_resetAgentData 000000018000916c     libiterreachobj002.obj
 0002:00003174       $unwind$MA_checkStatus     0000000180009174     libiterreachobj002.obj
 0002:00003188       $unwind$Java_nsk_jvmti_unit_FollowReferences_FollowRefObjects_setTag 0000000180009188     libiterreachobj002.obj
 0002:000031a0       $unwind$Java_nsk_jvmti_unit_FollowReferences_FollowRefObjects_addRefToVerify 00000001800091a0     libiterreachobj002.obj
 0002:000031bc       $unwind$heapRootCallbackForFirstObjectsIteration 00000001800091bc     libiterreachobj002.obj
 0002:000031bc       $unwind$objectReferenceCallbackForFirstObjectsIteration 00000001800091bc     libiterreachobj002.obj
 0002:000031bc       $unwind$stackReferenceCallbackForFirstObjectsIteration 00000001800091bc     libiterreachobj002.obj
 0002:000031d0       $unwind$heapRootCallbackForSecondObjectsIteration 00000001800091d0     libiterreachobj002.obj
 0002:000031d0       $unwind$objectReferenceCallbackForSecondObjectsIteration 00000001800091d0     libiterreachobj002.obj
 0002:000031d0       $unwind$stackReferenceCallbackForSecondObjectsIteration 00000001800091d0     libiterreachobj002.obj
 0002:000031e8       $unwind$capture_previous_context 00000001800091e8     MSVCRT:gs_report.obj
 0002:000031f4       $unwind$__GSHandlerCheckCommon 00000001800091f4     MSVCRT:gshandler.obj
 0002:00003200       $xdatasym                  0000000180009200     MSVCRT:amdsecgs.obj
 0002:00003204       $unwind$?dllmain_crt_process_attach@@YAHQEAUHINSTANCE__@@QEAX@Z 0000000180009204     MSVCRT:dll_dllmain.obj
 0002:00003240       $unwind$?fin$0@?0??dllmain_crt_process_attach@@YAHQEAUHINSTANCE__@@QEAX@Z@4HA 0000000180009240     MSVCRT:dll_dllmain.obj
 0002:00003240       $unwind$?fin$0@?0??dllmain_crt_process_detach@@YAH_N@Z@4HA 0000000180009240     MSVCRT:dll_dllmain.obj
 0002:00003240       $unwind$?fin$1@?0??dllmain_crt_process_detach@@YAH_N@Z@4HA 0000000180009240     MSVCRT:dll_dllmain.obj
 0002:00003248       $unwind$?dllmain_crt_process_detach@@YAH_N@Z 0000000180009248     MSVCRT:dll_dllmain.obj
 0002:0000329c       $unwind$?dllmain_dispatch@@YAHQEAUHINSTANCE__@@KQEAX@Z 000000018000929c     MSVCRT:dll_dllmain.obj
 0002:000032c4       $unwind$?filt$0@?0??dllmain_dispatch@@YAHQEAUHINSTANCE__@@KQEAX@Z@4HA 00000001800092c4     MSVCRT:dll_dllmain.obj
 0002:000032cc       $unwind$__scrt_is_nonwritable_in_current_image 00000001800092cc     MSVCRT:utility.obj
 0002:000032ec       $unwind$__scrt_is_nonwritable_in_current_image$filt$0 00000001800092ec     MSVCRT:utility.obj
 0002:000032f4       $unwind$__scrt_fastfail    00000001800092f4     MSVCRT:utility_desktop.obj
 0002:00003304       $unwind$__security_init_cookie 0000000180009304     MSVCRT:gs_support.obj
 0002:00003310       $unwind$__isa_available_init 0000000180009310     MSVCRT:cpu_disp.obj
 0002:00003320       $xdatasym                  0000000180009320     MSVCRT:guard_dispatch.obj
 0002:00003328       $xdatasym                  0000000180009328     MSVCRT:guard_xfg_dispatch.obj
 0002:00003330       .edata                     0000000180009330     iterreachobj002.exp
 0002:00003358       rgpv                       0000000180009358     iterreachobj002.exp
 0002:00003390       rgszName                   0000000180009390     iterreachobj002.exp
 0002:000033c8       rgwOrd                     00000001800093c8     iterreachobj002.exp
 0002:000033e4       szName                     00000001800093e4     iterreachobj002.exp
 0002:000033f8       $N00001                    00000001800093f8     iterreachobj002.exp
 0002:00003407       $N00002                    0000000180009407     iterreachobj002.exp
 0002:00003414       $N00003                    0000000180009414     iterreachobj002.exp
 0002:00003459       $N00004                    0000000180009459     iterreachobj002.exp
 0002:00003496       $N00005                    0000000180009496     iterreachobj002.exp
 0002:000034de       $N00006                    00000001800094de     iterreachobj002.exp
 0002:0000351e       $N00007                    000000018000951e     iterreachobj002.exp
 0002:0000355b       $N00008                    000000018000955b     iterreachobj002.exp
 0002:00003596       $N00009                    0000000180009596     iterreachobj002.exp
 0002:000035c4       $N00010                    00000001800095c4     iterreachobj002.exp
 0002:000035f5       $N00011                    00000001800095f5     iterreachobj002.exp
 0002:00003624       $N00012                    0000000180009624     iterreachobj002.exp
 0002:00003653       $N00013                    0000000180009653     iterreachobj002.exp
 0002:00003688       $N00014                    0000000180009688     iterreachobj002.exp
 0002:00003aea       .idata$6                   0000000180009aea     kernel32:KERNEL32.dll
 0002:00003b4e       .idata$6                   0000000180009b4e     vcruntime:VCRUNTIME140.dll
 0002:00003ce0       .idata$6                   0000000180009ce0     ucrt:api-ms-win-crt-heap-l1-1-0.dll
 0002:00003d00       .idata$6                   0000000180009d00     ucrt:api-ms-win-crt-runtime-l1-1-0.dll
 0002:00003d22       .idata$6                   0000000180009d22     ucrt:api-ms-win-crt-convert-l1-1-0.dll
 0002:00003d44       .idata$6                   0000000180009d44     ucrt:api-ms-win-crt-stdio-l1-1-0.dll
 0002:00003d64       .idata$6                   0000000180009d64     ucrt:api-ms-win-crt-string-l1-1-0.dll
 0003:00000000       ?codeAttributeName@@3PEBDEB 000000018000a000     libiterreachobj002.obj
 0003:00000008       ?lineNumberAttributeName@@3PEBDEB 000000018000a008     libiterreachobj002.obj
 0003:00000010       ?localVarAttributeName@@3PEBDEB 000000018000a010     libiterreachobj002.obj
 0003:00000018       ?localVarTypeAttributeName@@3PEBDEB 000000018000a018     libiterreachobj002.obj
 0003:00000020       ?stackMapAttributeName@@3PEBDEB 000000018000a020     libiterreachobj002.obj
 0003:00000028       ?callBytes@@3PAEA          000000018000a028     libiterreachobj002.obj
 0003:0000002c       ?allocBytes@@3PAEA         000000018000a02c     libiterreachobj002.obj
 0003:0001aad4       redefineAttempted          0000000180024ad4     libiterreachobj002.obj
 0003:0001aad8       nsk_context                0000000180024ad8     libiterreachobj002.obj
 0003:0001aae4       redefineSucceed            0000000180024ae4     libiterreachobj002.obj
 0003:0001aae8       agentFailed                0000000180024ae8     libiterreachobj002.obj
 0003:0001aaec       currentAgentStatus         0000000180024aec     libiterreachobj002.obj
 0003:0001aaf0       context                    0000000180024af0     libiterreachobj002.obj
 0003:0001aba8       agentThread                0000000180024ba8     libiterreachobj002.obj
 0003:0001abb0       agentThreadProc            0000000180024bb0     libiterreachobj002.obj
 0003:0001abb8       agentThreadArg             0000000180024bb8     libiterreachobj002.obj
 0003:0001abc0       agent_data                 0000000180024bc0     libiterreachobj002.obj
 0003:0001abd0       jvmti_env                  0000000180024bd0     libiterreachobj002.obj
 0003:0001abd8       jvm                        0000000180024bd8     libiterreachobj002.obj
 0003:0001abe0       jni_env                    0000000180024be0     libiterreachobj002.obj
 0003:0001abe8       checkStatus_func           0000000180024be8     libiterreachobj002.obj
 0003:0001abf0       ?codeAttributeIndex@@3GA   0000000180024bf0     libiterreachobj002.obj
 0003:0001abf4       ?lineNumberAttributeIndex@@3GA 0000000180024bf4     libiterreachobj002.obj
 0003:0001abf8       ?localVarAttributeIndex@@3GA 0000000180024bf8     libiterreachobj002.obj
 0003:0001abfc       ?localVarTypeAttributeIndex@@3GA 0000000180024bfc     libiterreachobj002.obj
 0003:0001ac00       ?stackMapAttributeIndex@@3GA 0000000180024c00     libiterreachobj002.obj
 0003:0001ac04       ?stackFrameOffset@@3GA     0000000180024c04     libiterreachobj002.obj
 0003:0001ac08       ?mode@@3HA                 0000000180024c08     libiterreachobj002.obj
 0003:0001ac0c       ?constantPoolSize@@3GA     0000000180024c0c     libiterreachobj002.obj
 0003:0001ac10       ?orig@@3PEBEEB             0000000180024c10     libiterreachobj002.obj
 0003:0001ac18       ?gen@@3PEAEEA              0000000180024c18     libiterreachobj002.obj
 0003:0001ac20       ?inputPos@@3PEAEEA         0000000180024c20     libiterreachobj002.obj
 0003:0001ac28       ?endPos@@3PEBEEB           0000000180024c28     libiterreachobj002.obj
 0003:0001ac30       ?genPos@@3PEAEEA           0000000180024c30     libiterreachobj002.obj
 0003:0001ac38       ?markPos@@3PEAEEA          0000000180024c38     libiterreachobj002.obj
 0003:0001ac40       ?constantPool@@3PEAPEADEA  0000000180024c40     libiterreachobj002.obj
 0003:0001ac48       ?constantPoolCount@@3GA    0000000180024c48     libiterreachobj002.obj
 0003:0001ac4c       ?zeroBytes@@3PAEA          0000000180024c4c     libiterreachobj002.obj
 0003:0001ac50       ?codeLength@@3IA           0000000180024c50     libiterreachobj002.obj
 0003:0001ac54       objectCount                0000000180024c54     libiterreachobj002.obj
 0003:0001ac58       ?map@@3PEAIEA              0000000180024c58     libiterreachobj002.obj
 0003:0001ac60       ?widening@@3PEACEA         0000000180024c60     libiterreachobj002.obj
 0003:0001ac68       jvmti                      0000000180024c68     libiterreachobj002.obj
 0003:0001ac70       callbacks                  0000000180024c70     libiterreachobj002.obj
 0003:0001ada8       caps                       0000000180024da8     libiterreachobj002.obj
 0003:0001adb8       timeout                    0000000180024db8     libiterreachobj002.obj
 0003:0001adc0       objectCountMax             0000000180024dc0     libiterreachobj002.obj
 0003:0001adc4       userData                   0000000180024dc4     libiterreachobj002.obj
 0003:0001adc8       callbackAborted            0000000180024dc8     libiterreachobj002.obj
 0003:0001adcc       numberOfDeallocatedFromCallbacksDescriptors 0000000180024dcc     libiterreachobj002.obj
 0003:0001add0       objectDescList             0000000180024dd0     libiterreachobj002.obj
 0003:0001add8       objectDescListStart        0000000180024dd8     libiterreachobj002.obj
 0003:0001ade0       objectDescBuf              0000000180024de0     libiterreachobj002.obj
 0003:0001ade8       objectDescArr              0000000180024de8     libiterreachobj002.obj
 0003:0001adf0       deallocatedFlagsArr        0000000180024df0     libiterreachobj002.obj
 0003:0001ae00       GS_ExceptionRecord         0000000180024e00     MSVCRT:gs_report.obj
 0003:0001aea0       GS_ContextRecord           0000000180024ea0     MSVCRT:gs_report.obj
 0003:0001b370       ?g_tss_cv@@3U_RTL_CONDITION_VARIABLE@@A 0000000180025370     MSVCRT:thread_safe_statics.obj
 0003:0001b378       ?g_tss_event@@3PEAXEA      0000000180025378     MSVCRT:thread_safe_statics.obj
 0003:0001b380       ?g_tss_mutex@@3U_RTL_CRITICAL_SECTION@@A 0000000180025380     MSVCRT:thread_safe_statics.obj
 0003:0001b3a8       ?g_sleep_condition_variable_cs@@3P6AHPEAU_RTL_CONDITION_VARIABLE@@PEAU_RTL_CRITICAL_SECTION@@K@ZEA 00000001800253a8     MSVCRT:thread_safe_statics.obj
 0003:0001b3b0       ?g_wake_all_condition_variable@@3P6AXPEAU_RTL_CONDITION_VARIABLE@@@ZEA 00000001800253b0     MSVCRT:thread_safe_statics.obj
 0003:0001b3bc       ?__proc_attached@@3HA      00000001800253bc     MSVCRT:dll_dllmain.obj
 0003:0001b3d0       ?is_initialized_as_dll@@3_NA 00000001800253d0     MSVCRT:utility.obj
 0003:0001b3d1       ?module_local_atexit_table_initialized@@3_NA 00000001800253d1     MSVCRT:utility.obj
 0003:0001b3d8       ?module_local_atexit_table@@3U_onexit_table_t@@A 00000001800253d8     MSVCRT:utility.obj
 0003:0001b3f0       ?module_local_at_quick_exit_table@@3U_onexit_table_t@@A 00000001800253f0     MSVCRT:utility.obj
